:020000040000FA
:1000000000000000000000000000000000000000F0
:1000100000000000000000000000000000000000E0
:1000200000000000000000000000000000000000D0
:1000300000000000000000000000000000000000C0
:1000400000000000000000000000000000000000B0
:1000500000000000000000000000000000000000A0
:100060000000000000000000000000000000000090
:100070000000000000000000000000000000000080
:100080000000000000000000000000000000000070
:100090000000000000000000000000000000000060
:1000A0000000000000000000000000000000000050
:1000B0000000000000000000000000000000000040
:1000C0000000000000000000000000000000000030
:1000D0000000000000000000000000000000000020
:1000E0000000000000000000000000000000000010
:1000F0000000000000000000000000000000000000
:1001000000000000000000000000000000000000EF
:1001100000000000000000000000000000000000DF
:1001200000000000000000000000000000000000CF
:1001300000000000000000000000000000000000BF
:1001400000000000000000000000000000000000AF
:10015000000000000000000000000000000000009F
:10016000000000000000000000000000000000008F
:10017000000000000000000000000000000000007F
:10018000000000000000000000000000000000006F
:10019000000000000000000000000000000000005F
:1001A000000000000000000000000000000000004F
:1001B000000000000000000000000000000000003F
:1001C000000000000000000000000000000000002F
:1001D000000000000000000000000000000000001F
:1001E000000000000000000000000000000000000F
:1001F00000000000000000000000000000000000FF
:10020000EE6A010FD8A400EF01F00EEE00F0000E30
:10021000EE6A010FD8A408EF01F01DEE00F02DEEFC
:1002200000F0F86A240EAC6E0C0EAF6E900EAB6E42
:10023000AB980000AB88AE50AE50240E6C6E0C0E26
:100240006F6E900E6B6E6B9800006B886E506E50E8
:100250003F0E40DFFA0E57EC01F0FA0E57EC01F0BA
:10026000FA0E57EC01F0FA0E57EC01F0A4AA04D0F4
:1002700035DF5508D8B4D1D686EC01F02C6E2CB001
:1002800002D0BED2CAD63F0E25DFFA0E57EC01F0DF
:10029000FA0E57EC01F0FA0E57EC01F0FA0E57EC9B
:1002A00001F09EAAF0D71ADF5508ECE0ECD7266ED5
:1002B000060E276E286A0400282EFDD7272EFAD7AF
:1002C000262EF6D71200FB0EE3CFF6FFFC0EE3CF8F
:1002D000F7FFFD0EE3CFF8FFFE0EE3CFE9FFFF0EC1
:1002E000E3CFEAFFE9CFF3FFEACFF4FFF90EE350E3
:1002F00003E1FA0EE35009E0F90EE30602E2FA0E1A
:10030000E3060900F5CFEEFFF1D71200D9CFE6FFE3
:10031000DACFE6FFE1CFD9FFE2CFDAFF0C0EE1241E
:1003200002E3E168E652E16E050EDB6A060EDB6A67
:10033000090EDB6A080EF36E0A0EF3CFDBFF0B0E1D
:10034000DB6ADE6A080EDE6EDE6ADD6ADD52DD52D1
:10035000D9CFE9FFDACFEAFFD880FE0EEE54FF0EC8
:10036000EE54010EEE54000EEE546BE30400050E45
:10037000DBCF00F0060EDBCF01F001C000F0016A18
:10038000090EDBCFF6FF0A0EDBCFF7FF0B0EDBCF3C
:10039000F8FF0800F5500018E76E040EE7CFDBFF0A
:1003A000020EE66EE66A040E016ADB34FE0B0136CD
:1003B000006EF00E0026050E0122026A00C0E6FF64
:1003C00001C0E6FF02C0E6FFD950070FE66E000E3F
:1003D000DA20E66E63EC01F0F56E070EE15C02E2F6
:1003E000E16AE552E16EF550050EDBCF02F002C086
:1003F00003F0026A000E0216FF0E0316070EDB5012
:100400000218006E080EDB500318016E050E00C0C6
:10041000DBFF060E01C0DBFFD950090FE96E000EAD
:10042000DA20EA6EEE2A000EEE22000EEE22D9CF7E
:10043000E9FFDACFEAFFEE2A000EEE22EE22EE22EC
:1004400087D7050EDBCF00F0060EDBCF01F001C031
:1004500000F0016AD950090FE96E000EDA20EA6E49
:10046000EFCFF6FFEE2AEFCFF7FF000EEE22EFCF31
:10047000F8FF000EEE220800F550005C14E1090EB2
:10048000DBCFF6FF0A0EDBCFF7FF0B0EDBCFF8FF5B
:100490000800F550F36E050EDB50F35C02E1000E30
:1004A00001D0010E01D0010EF56E0C0EE15C02E2EE
:1004B000E16AE552E16EF550E552E5CFDAFFE7CFAC
:1004C000D9FF1200FF00FF00FF00FF00FF00FF0048
:1004D000FF00FF00FF00FF00FF00FF00FF00FF0024
:1004E000FF00FF00FF00FF00FF00FF00FF00FF0014
:1004F000FF00FF00FF00FF00FF00FF00FF00FF0004
:10050000FF00FF00FF00FF00FF00FF00FF00FF00F3
:10051000FF00FF00FF00FF00FF00FF00FF00FF00E3
:10052000FF00FF00FF00FF00FF00FF00FF00FF00D3
:10053000FF00FF00FF00FF00FF00FF00FF00FF00C3
:10054000FF00FF00FF00FF00FF00FF00FF00FF00B3
:10055000FF00FF00FF00FF00FF00FF00FF00FF00A3
:10056000FF00FF00FF00FF00FF00FF00FF00FF0093
:10057000FF00FF00FF00FF00FF00FF00FF00FF0083
:10058000FF00FF00FF00FF00FF00FF00FF00FF0073
:10059000FF00FF00FF00FF00FF00FF00FF00FF0063
:1005A000FF00FF00FF00FF00FF00FF00FF00FF0053
:1005B000FF00FF00FF00FF00FF00FF00FF00FF0043
:1005C000FF00FF00FF00FF00FF00FF00FF00FF0033
:1005D000FF00FF00FF00FF00FF00FF00FF00FF0023
:1005E000FF00FF00FF00FF00FF00FF00FF00FF0013
:1005F00000002110422063308440A550C660E7709F
:10060000088129914AA16BB18CC1ADD1CEE1EFF146
:100610003112100273325222B5529442F772D662EE
:10062000399318837BB35AA3BDD39CC3FFF3DEE396
:100630006224433420040114E664C774A44485543E
:100640006AA54BB528850995EEE5CFF5ACC58DD5E6
:100650005336722611163006D776F6669556B4468E
:100660005BB77AA719973887DFF7FEE79DD7BCC736
:10067000C448E5588668A7784008611802282338DE
:10068000CCC9EDD98EE9AFF9488969990AA92BB986
:10069000F55AD44AB77A966A711A500A333A122A2E
:1006A000FDDBDCCBBFFB9EEB799B588B3BBB1AABD6
:1006B000A66C877CE44CC55C222C033C600C411C7E
:1006C000AEED8FFDECCDCDDD2AAD0BBD688D499D26
:1006D000977EB66ED55EF44E133E322E511E700ECE
:1006E0009FFFBEEFDDDFFCCF1BBF3AAF599F788F76
:1006F0008891A981CAB1EBA10CD12DC14EF16FE156
:100700008010A100C230E32004502540467067608D
:10071000B9839893FBA3DAB33DC31CD37FE35EF3A5
:10072000B1029012F322D2323542145277625672DD
:10073000EAB5CBA5A89589856EF54FE52CD50DC5F5
:10074000E234C324A014810466744764245405442D
:10075000DBA7FAB79987B8975FE77EF71DC73CD745
:10076000D326F2369106B01657667676154634567D
:100770004CD96DC90EF92FE9C899E9898AB9ABA995
:100780004458654806782768C018E1088238A328CD
:100790007DCB5CDB3FEB1EFBF98BD89BBBAB9ABBE5
:1007A000754A545A376A167AF10AD01AB32A923A1D
:1007B0002EFD0FED6CDD4DCDAABD8BADE89DC98D35
:1007C000267C076C645C454CA23C832CE01CC10C6D
:1007D0001FEF3EFF5DCF7CDF9BAFBABFD98FF89F85
:1007E000176E367E554E745E932EB23ED10EF01EBD
:1007F00001010000FF00FF00FF00FF00FF00FF00FD
:10080000FBEF51F01200FF009BEF3AF01200FF00E7
:10081000FF00FF00FF00FF00FF00FF00FF00FF00E0
:10082000FF00FF00FF00FF00FF00FF00FF00FF00D0
:1008300006005EA400001002000010000000A1608D
:100840000000FE010000010000005AA40000EF0EAD
:1008500000000400000042A40000D70E00001800B1
:10086000000032A4000000020000100000002CA4D0
:1008700000004502000006000000270EE66E7C0E18
:10088000E66EFBEC4FF0E552E5520C0EE66E3C0EC8
:10089000E66EC9EC4FF0E552E55284900000849278
:1008A0000101F26B1200D9CFE6FFDACFE6FFE1CF0C
:1008B000D9FFE2CFDAFFFC0EDBCFE9FFFD0EDBCF85
:1008C000EAFFEF5011E06CA2FED7FC0EDBCFE9FF90
:1008D000DB2AFD0EDBCFEAFF01E3DB2AEF50E66EF9
:1008E00074EC51F0E552E7D7E552E5CFDAFFE7CFF8
:1008F000D9FF1200D9CFE6FFDACFE6FFE1CFD9FF6B
:10090000E2CFDAFFFC0EDBCFF6FFFD0EDBCFF7FF09
:100910000800F55012E06CA2FED7FC0EDBCFF6FF0C
:10092000DB2AFD0EDBCFF7FF01E3DB2A0800F550E1
:10093000E66E74EC51F0E552E5D7E552E5CFDAFF0B
:10094000E7CFD9FF1200D9CFE6FFDACFE6FFE1CF3C
:10095000D9FFE2CFDAFF848000008482FB0EDBCF78
:10096000F3FFDB06F350000911E0ACA2FED7FC0E4A
:10097000DBCFE9FFDB2AFD0EDBCFEAFF01E3DB2A59
:10098000EF50E66E8BEC51F0E552E8D7ACA2FED703
:10099000849000008492E552E5CFDAFFE7CFD9FFDB
:1009A0001200D9CFE6FFDACFE6FFE1CFD9FFE2CFE1
:1009B000DAFF848000008482FD0EDBCFE6FF8BEC43
:1009C00051F0E552ACA2FED7849000008492E5522B
:1009D000E5CFDAFFE7CFD9FF1200D9CFE6FFDACFB4
:1009E000E6FFE1CFD9FFE2CFDAFFE6520101815104
:1009F0003F0802E20101816B9D9A01018151812B27
:100A0000EA6A400FE96E010EEA22EFCFDFFF9D8A0E
:100A1000DF5000D0E552E552E5CFDAFFE7CFD9FF4E
:100A20001200D9CFE6FFDACFE6FFE1CFD9FFE2CF60
:100A3000DAFFE652E6529D9A010E80C1DBFF9D8AE5
:100A4000010EDB500101D880815506E3010EDB5019
:100A50000101D8808155DF6E01018151F36E010ED5
:100A6000DBCFF4FFF350F45C0AE2010EDBCFE6FFCC
:100A7000400E0101D8808155E552E724DF6EDF503A
:100A800000D0E552E552E552E5CFDAFFE7CFD9FFD6
:100A90001200D9CFE6FFDACFE6FFE1CFD9FFE2CFF0
:100AA000DAFF8480000084820101C2513F0802E223
:100AB0000101C26B0101C251C22BEA6A820FE96EC9
:100AC000010EEA22FD0EDBCFEFFFE552E5CFDAFFA4
:100AD000E7CFD9FF12000101806B0101816B010199
:100AE000C26B0101C36B1200D9CFE6FFDACFE6FF7C
:100AF000E1CFD9FFE2CFDAFFE652E652FC0EDBCFC0
:100B0000E9FFDB2AFD0EDBCFEAFF01E3DB2A010E62
:100B1000EFCFDBFFFC0EDBCFE9FFFD0EDBCFEAFF03
:100B2000EFCFDFFFDECF00F0DDCF01F000C0F3FF3D
:100B300001C0F4FF00D0E552E552E552E5CFDAFFFF
:100B4000E7CFD9FF1200D9CFE6FFDACFE6FFE1CF3A
:100B5000D9FFE2CFDAFF070EE12402E3E168E652B3
:100B6000E16E050E0101EC5D02E067EF0DF0060E8F
:100B7000DB6A040EDB6A050EDB6A040EDBCF00F0D5
:100B8000050EDBCF01F00101EE51000101AE02D0F4
:100B9000D89003D0005C000E015818E2040EDBCFA1
:100BA000E9FF050EDBCFEAFFC40EE926010EEA22BB
:100BB000060EDBCFE7FFEF50E726060EE7CFDBFFA1
:100BC000040EDB2A050E01E3DB2AD7D7060EDB5025
:100BD00002E064EF0DF00101C851480A02E157EF4D
:100BE0000BF0110A01E1FCD11A0A01E151D1020A0C
:100BF00001E10AD1030A01E1B2D0080A4DE0030A7B
:100C00000BE0130A02E012EF0DF00101060EC46FB3
:100C10000101C56B18EF0DF00101060EC46F010153
:100C2000100EC56F88CE00F0016A00C0C6F187CEF5
:100C3000C7F18ACE00F0016A00C0C8F189CEC9F1BF
:100C40008CCE00F0016A00C0CAF18BCECBF18ECE03
:100C500000F0016A00C0CCF18DCECDF190CE00F055
:100C6000016A00C0CEF18FCECFF194CE00F0016AC0
:100C700000C0D0F193CED1F192CE00F0016A00C055
:100C8000D2F191CED3F196CE00F0016A00C0D4F13A
:100C900095CED5F118EF0DF0C90EE66E010EE66E99
:100CA00023DFE552E552F3CF87FEF4CF88FECB0E6B
:100CB000E66E010EE66E18DFE552E552F3CF89FECF
:100CC000F4CF8AFECD0EE66E010EE66E0DDFE55224
:100CD000E552F3CF8BFEF4CF8CFECF0EE66E010E05
:100CE000E66E02DFE552E552F3CF8DFEF4CF8EFEC5
:100CF000D10EE66E010EE66EF7DEE552E552F3CF59
:100D00008FFEF4CF90FED30EE66E010EE66EECDEA3
:100D1000E552E552F3CF93FEF4CF94FED50EE66E86
:100D2000010EE66EE1DEE552E552F3CF91FEF4CF1F
:100D300092FED70EE66E010EE66ED6DEE552E55265
:100D4000F3CF95FEF4CF96FE14EC12F0D0EC0EF03B
:100D50000101060EC46F0101C56B18EF0DF0010112
:100D6000C951310A26E0010A01E046D00101060E10
:100D7000C46F0101040EC56F31C202F032C203F02C
:100D80000001046A056A03C000F0016A00C0C6F1F0
:100D900031C200F032C201F00001026A036A00C0F1
:100DA000C7F130C200F0016A00C0C8F12FC2C9F11A
:100DB00029D00101060EC46F0101040EC56F35C2B2
:100DC00002F036C203F00001046A056A03C000F0B5
:100DD000016A00C0C6F135C200F036C201F0000160
:100DE000026A036A00C0C7F134C200F0016A00C0A1
:100DF000C8F133C2C9F106D00101150EC46F01015B
:100E0000C56B00D018EF0DF00101C951300A01E0A7
:100E100037D00101060EC46F0101040EC56FF00E3C
:100E2000F66EF768010EF86E0900F5CF00F00800C5
:100E3000F5CF01F001C000F0016A00C0C6F1F00E6C
:100E4000F66EF768010EF86E0800F5CFC7F1F20EE6
:100E5000F66EF768010EF86E0900F5CF00F0080095
:100E6000F5CF01F001C000F0016A00C0C8F1F20E38
:100E7000F66EF768010EF86E0800F5CFC9F106D0DE
:100E80000101150EC46F0101C56B00D018EF0DF004
:100E90000101C951300A01E09BD00101060EC46F67
:100EA0000101040EC56FDE6ADE6ADE6ADD6ADD52AC
:100EB000DD520E010C5106E0D9CFE9FFDACFEAFF8F
:100EC000EE52EE820E01065106E0D9CFE9FFDACFED
:100ED000EAFFEE52EE800E01365105E0D9CFE9FF70
:100EE000DACFEAFFEE8E0E013C5105E0D9CFE9FFE3
:100EF000DACFEAFFEE8C0E01305105E0D9CFE9FFE1
:100F0000DACFEAFFEE8A0E012A5105E0D9CFE9FFD8
:100F1000DACFEAFFEE880E01245105E0D9CFE9FFD0
:100F2000DACFEAFFEE860E011E5105E0D9CFE9FFC8
:100F3000DACFEAFFEE840E01185105E0D9CFE9FFC0
:100F4000DACFEAFFEE820E01125105E0D9CFE9FFB8
:100F5000DACFEAFFEE80D9CFE9FFDACFEAFFEECFB2
:100F600002F0EECF03F0EECF04F0EFCF05F0100E5D
:100F7000D8900532043203320232E806F9E103C0A8
:100F800000F0016A00C0C6F1D9CFE9FFDACFEAFF6D
:100F9000EECF00F0EECF01F0EECF02F0EFCF03F096
:100FA000100ED8900332023201320032E806F9E125
:100FB00000C0C7F1DFCF00F0010EDBCF01F001C0B0
:100FC00000F0016A00C0C8F1000EDBCFC9F106D005
:100FD0000101150EC46F0101C56B00D018EF0DF0B3
:100FE0000101060EC46F0101240EC56F006A016A7B
:100FF0007A0E026E440E036EB9CE37F0BACE38F0D8
:10100000BBCE39F0BCCE3AF000C032F001C033F0B4
:1010100002C034F003C035F0B6EC3DF0EAEC3EF02F
:1010200031C0DEFF32C0DEFF33C0DEFF34C0DDFF83
:10103000DD52DD52D9CFE9FFDACFEAFFEECF02F081
:10104000EECF03F0EECF04F0EFCF05F0100ED89006
:101050000532043203320232E806F9E103C000F03F
:10106000016A00C0C6F1D9CFE9FFDACFEAFFEECFBF
:1010700000F0EECF01F0EECF02F0EFCF03F0100E54
:10108000D8900332023201320032E806F9E100C0A2
:10109000C7F1DFCF00F0010EDBCF01F001C000F09F
:1010A000016A00C0C8F1000EDBCFC9F1006A016A15
:1010B0007A0E026E440E036EBDCE37F0BECE38F00F
:1010C000BFCE39F0C0CE3AF000C032F001C033F0EC
:1010D00002C034F003C035F0B6EC3DF0EAEC3EF06F
:1010E00031C0DEFF32C0DEFF33C0DEFF34C0DDFFC3
:1010F000DD52DD52D9CFE9FFDACFEAFFEECF02F0C1
:10110000EECF03F0EECF04F0EFCF05F0100ED89045
:101110000532043203320232E806F9E103C000F07E
:10112000016A00C0CAF1D9CFE9FFDACFEAFFEECFFA
:1011300000F0EECF01F0EECF02F0EFCF03F0100E93
:10114000D8900332023201320032E806F9E100C0E1
:10115000CBF1DFCF00F0010EDBCF01F001C000F0DA
:10116000016A00C0CCF1000EDBCFCDF1006A016A4C
:101170007A0E026E440E036EC1CE37F0C2CE38F046
:10118000C3CE39F0C4CE3AF000C032F001C033F023
:1011900002C034F003C035F0B6EC3DF0EAEC3EF0AE
:1011A00031C0DEFF32C0DEFF33C0DEFF34C0DDFF02
:1011B000DD52DD52D9CFE9FFDACFEAFFEECF02F000
:1011C000EECF03F0EECF04F0EFCF05F0100ED89085
:1011D0000532043203320232E806F9E103C000F0BE
:1011E000016A00C0CEF1D9CFE9FFDACFEAFFEECF36
:1011F00000F0EECF01F0EECF02F0EFCF03F0100ED3
:10120000D8900332023201320032E806F9E100C020
:10121000CFF1DFCF00F0010EDBCF01F001C000F015
:10122000016A00C0D0F1000EDBCFD1F1006A016A83
:101230007A0E026E440E036E99CE37F09ACE38F0D5
:101240009BCE39F09CCE3AF000C032F001C033F0B2
:1012500002C034F003C035F0B6EC3DF0EAEC3EF0ED
:1012600031C0DEFF32C0DEFF33C0DEFF34C0DDFF41
:10127000DD52DD52D9CFE9FFDACFEAFFEECF02F03F
:10128000EECF03F0EECF04F0EFCF05F0100ED890C4
:101290000532043203320232E806F9E103C000F0FD
:1012A000016A00C0D2F1D9CFE9FFDACFEAFFEECF71
:1012B00000F0EECF01F0EECF02F0EFCF03F0100E12
:1012C000D8900332023201320032E806F9E100C060
:1012D000D3F1DFCF00F0010EDBCF01F001C000F051
:1012E000016A00C0D4F1000EDBCFD5F1006A016ABB
:1012F0007A0E026E440E036E9DCE37F09ECE38F00D
:101300009FCE39F0A0CE3AF000C032F001C033F0E9
:1013100002C034F003C035F0B6EC3DF0EAEC3EF02C
:1013200031C0DEFF32C0DEFF33C0DEFF34C0DDFF80
:10133000DD52DD52D9CFE9FFDACFEAFFEECF02F07E
:10134000EECF03F0EECF04F0EFCF05F0100ED89003
:101350000532043203320232E806F9E103C000F03C
:10136000016A00C0D6F1D9CFE9FFDACFEAFFEECFAC
:1013700000F0EECF01F0EECF02F0EFCF03F0100E51
:10138000D8900332023201320032E806F9E100C09F
:10139000D7F1DFCF00F0010EDBCF01F001C000F08C
:1013A000016A00C0D8F1000EDBCFD9F1006A016AF2
:1013B0007A0E026E440E036EA1CE37F0A2CE38F044
:1013C000A3CE39F0A4CE3AF000C032F001C033F021
:1013D00002C034F003C035F0B6EC3DF0EAEC3EF06C
:1013E00031C0DEFF32C0DEFF33C0DEFF34C0DDFFC0
:1013F000DD52DD52D9CFE9FFDACFEAFFEECF02F0BE
:10140000EECF03F0EECF04F0EFCF05F0100ED89042
:101410000532043203320232E806F9E103C000F07B
:10142000016A00C0DAF1D9CFE9FFDACFEAFFEECFE7
:1014300000F0EECF01F0EECF02F0EFCF03F0100E90
:10144000D8900332023201320032E806F9E100C0DE
:10145000DBF1DFCF00F0010EDBCF01F001C000F0C7
:10146000016A00C0DCF1000EDBCFDDF1006A016A29
:101470007A0E026E440E036EA5CE37F0A6CE38F07B
:10148000A7CE39F0A8CE3AF000C032F001C033F058
:1014900002C034F003C035F0B6EC3DF0EAEC3EF0AB
:1014A00031C0DEFF32C0DEFF33C0DEFF34C0DDFFFF
:1014B000DD52DD52D9CFE9FFDACFEAFFEECF02F0FD
:1014C000EECF03F0EECF04F0EFCF05F0100ED89082
:1014D0000532043203320232E806F9E103C000F0BB
:1014E000016A00C0DEF1D9CFE9FFDACFEAFFEECF23
:1014F00000F0EECF01F0EECF02F0EFCF03F0100ED0
:10150000D8900332023201320032E806F9E100C01D
:10151000DFF1DFCF00F0010EDBCF01F001C000F002
:10152000016A00C0E0F1000EDBCFE1F1006A016A60
:101530007A0E026E440E036EB5CE37F0B6CE38F09A
:10154000B7CE39F0B8CE3AF000C032F001C033F077
:1015500002C034F003C035F0B6EC3DF0EAEC3EF0EA
:1015600031C0DEFF32C0DEFF33C0DEFF34C0DDFF3E
:10157000DD52DD52D9CFE9FFDACFEAFFEECF02F03C
:10158000EECF03F0EECF04F0EFCF05F0100ED890C1
:101590000532043203320232E806F9E103C000F0FA
:1015A000016A00C0E2F1D9CFE9FFDACFEAFFEECF5E
:1015B00000F0EECF01F0EECF02F0EFCF03F0100E0F
:1015C000D8900332023201320032E806F9E100C05D
:1015D000E3F1DFCF00F0010EDBCF01F001C000F03E
:1015E000016A00C0E4F1000EDBCFE5F1006A016A98
:1015F0007A0E026E440E036EB1CE37F0B2CE38F0E2
:10160000B3CE39F0B4CE3AF000C032F001C033F0BE
:1016100002C034F003C035F0B6EC3DF0EAEC3EF029
:1016200031C0DEFF32C0DEFF33C0DEFF34C0DDFF7D
:10163000DD52DD52D9CFE9FFDACFEAFFEECF02F07B
:10164000EECF03F0EECF04F0EFCF05F0100ED89000
:101650000532043203320232E806F9E103C000F039
:10166000016A00C0E6F1D9CFE9FFDACFEAFFEECF99
:1016700000F0EECF01F0EECF02F0EFCF03F0100E4E
:10168000D8900332023201320032E806F9E100C09C
:10169000E7F1DFCF00F0010EDBCF01F001C000F079
:1016A000016A00C0E8F1000EDBCFE9F1C1D1300ED4
:1016B0000101C95D01E2AFD10101C951380801E260
:1016C000AAD10101C951380A01E13DD10F0A01E156
:1016D00015D1010A01E1EDD0030A01E1C5D0010AEB
:1016E00001E19DD0070A76E0010A4FE0030A28E0F5
:1016F000010A01E04DD1006A016A7A0E026E440EC1
:10170000036EB9CE37F0BACE38F0BBCE39F0BCCECE
:101710003AF000C032F001C033F002C034F003C030
:1017200035F0B6EC3DF0EAEC3EF031C0DEFF32C001
:10173000DEFF33C0DEFF34C0DDFFDD52DD5228D1D5
:10174000006A016A7A0E026E440E036EBDCE37F057
:10175000BECE38F0BFCE39F0C0CE3AF000C032F085
:1017600001C033F002C034F003C035F0B6EC3DF0F8
:10177000EAEC3EF031C0DEFF32C0DEFF33C0DEFFF8
:1017800034C0DDFFDD52DD5203D1006A016A7A0EFA
:10179000026E440E036EC1CE37F0C2CE38F0C3CE17
:1017A00039F0C4CE3AF000C032F001C033F002C0CC
:1017B00034F003C035F0B6EC3DF0EAEC3EF031C059
:1017C000DEFF32C0DEFF33C0DEFF34C0DDFFDD529E
:1017D000DD52DED0006A016A7A0E026E440E036E9C
:1017E00099CE37F09ACE38F09BCE39F09CCE3AF0B5
:1017F00000C032F001C033F002C034F003C035F055
:10180000B6EC3DF0EAEC3EF031C0DEFF32C0DEFF68
:1018100033C0DEFF34C0DDFFDD52DD52B9D0006AD7
:10182000016A7A0E026E440E036E9DCE37F09ECE94
:1018300038F09FCE39F0A0CE3AF000C032F001C0AF
:1018400033F002C034F003C035F0B6EC3DF0EAEC02
:101850003EF031C0DEFF32C0DEFF33C0DEFF34C0F9
:10186000DDFFDD52DD5294D0006A016A7A0E026E0D
:10187000440E036EA1CE37F0A2CE38F0A3CE39F0DD
:10188000A4CE3AF000C032F001C033F002C034F010
:1018900003C035F0B6EC3DF0EAEC3EF031C0DEFFBF
:1018A00032C0DEFF33C0DEFF34C0DDFFDD52DD526B
:1018B0006FD0006A016A7A0E026E440E036EA5CEE6
:1018C00037F0A6CE38F0A7CE39F0A8CE3AF000C057
:1018D00032F001C033F002C034F003C035F0B6EC92
:1018E0003DF0EAEC3EF031C0DEFF32C0DEFF33C037
:1018F000DEFF34C0DDFFDD52DD524AD0006A016AEE
:101900007A0E026E440E036EB5CE37F0B6CE38F0C6
:10191000B7CE39F0B8CE3AF000C032F001C033F0A3
:1019200002C034F003C035F0B6EC3DF0EAEC3EF016
:1019300031C0DEFF32C0DEFF33C0DEFF34C0DDFF6A
:10194000DD52DD5225D0006A016A7A0E026E440E25
:10195000036EB1CE37F0B2CE38F0B3CE39F0B4CE9C
:101960003AF000C032F001C033F002C034F003C0DE
:1019700035F0B6EC3DF0EAEC3EF031C0DEFF32C0AF
:10198000DEFF33C0DEFF34C0DDFFDD52DD5200D0AC
:101990000101060EC46F0101040EC56FD9CFE9FF26
:1019A000DACFEAFFEECF02F0EECF03F0EECF04F095
:1019B000EFCF05F0100ED890053204320332023218
:1019C000E806F9E103C000F0016A00C0C6F1D9CF12
:1019D000E9FFDACFEAFFEECF00F0EECF01F0EECF75
:1019E00002F0EFCF03F0100ED89003320232013232
:1019F0000032E806F9E100C0C7F1DFCF00F0010EC8
:101A0000DBCF01F001C000F0016A00C0C8F1000E98
:101A1000DBCFC9F106D00101150EC46F0101C56B02
:101A200007D006D00101150EC46F0101C56B00D0AF
:101A3000020E0101C5250101F06F0101030EEF6FD8
:101A4000060EDB6A040EDB6A050EDB6A040EDBCFD2
:101A500000F0050EDBCF01F00101F051000101AEF5
:101A600002D0D89003D0005C000E015818E2040E9A
:101A7000DBCFE9FF050EDBCFEAFFC40EE926010E3E
:101A8000EA22060EDBCFE7FFEF50E726060EE7CF90
:101A9000DBFF040EDB2A050E01E3DB2AD7D70101A9
:101AA000F02B060EDB50FF0DF350E66E0101F00542
:101AB000EA6AC40FE96E010EEA22E552E750EF6EC2
:101AC0000101060EEC6F02D00101EC6BE9D0060EAD
:101AD0000101EC5D31E10101EF512DE1040EDB6A02
:101AE000050EDB6A040EDBCF00F0050EDBCF01F044
:101AF0000101F051000101AE02D0D89003D0005C8A
:101B0000000E015815E2040EDBCFE9FF050EDBCF16
:101B1000EAFFC40EE926010EEA22EF50E66E49EC18
:101B200005F0E552040EDB2A050E01E3DB2ADAD7C5
:101B30009D880101EC6BB4D00101F15105E1010177
:101B4000EC5102E00101EC6B11EC05F0000901E140
:101B5000A7D0EDEC04F0E66ED950040FE96E000E4C
:101B6000DA20EA6EE552E750EE6EED6A0101EC51C3
:101B7000040A01E177D0070A59E0010A3BE0030AB1
:101B80001CE0010A01E089D0040EDBCFC4F10101A1
:101B9000010EED6FD950040FE96E000EDA20EA6EE7
:101BA000400EEE1801E1ED5007E10101010EEC6F6E
:101BB0000101FA0EF16F00D073D00101ED51ED2B50
:101BC000EA6AC40FE96E010EEA22040EDBCFEFFFD2
:101BD000D950040FE96E000EDA20EA6E420EEE18BC
:101BE00001E1ED5004E10101020EEC6F02D00101B0
:101BF000EC6B56D00101ED51EA6AC40FE96E010E9B
:101C0000EA22040EDBCFEFFF0101ED51ED2BEA6A72
:101C1000C40FE96E010EEA22EF50300804E1010121
:101C2000030EEC6F02D00101EC6B3AD0040EDB50D6
:101C3000230815E30101ED51ED2BEA6AC40FE96EAB
:101C4000010EEA22040EDBCFEFFF040EDB50040F7F
:101C5000010F0101EE6F0101040EEC6F02D00101D2
:101C6000EC6B1ED00101ED51ED2BEA6AC40FE96E59
:101C7000010EEA22040EDBCFEFFF0101EE5101015C
:101C8000ED5D04E30101050EEC6F06D0280E0101A5
:101C9000ED5D02E30101EC6B03D00101EC6B00D0C0
:101CA000F56E070EE15C02E2E16AE552E16EF55085
:101CB000E552E5CFDAFFE7CFD9FF1200730E006ED1
:101CC0005F0E016E026A00C0E6FF01C0E6FF7AEC1B
:101CD00004F0E552E552D2D9F3CF00F0F4CF01F091
:101CE000005001100BE1020EE66EE66AE66AE66A53
:101CF00073EC49F0E552E552E552E55251D801D86E
:101D000012000E01996B9A6B9B6B9C6B0E019D6B85
:101D10009E6B9F6BA06B0E01A16BA26BA36BA46B60
:101D20000E01A56BA66BA76BA86B0E01A96BAA6B26
:101D3000AB6BAC6B0E01B56BB66BB76BB86B0E01D2
:101D4000B16BB26BB36BB46B0E01C16BC26BC36B87
:101D5000C46B0E01AD6BAE6BAF6BB06B1200DBCE24
:101D600087FEDCCE88FEDDCE89FEDECE8AFEDFCEAB
:101D70008BFEE0CE8CFEE1CE8DFEE2CE8EFEE3CE7B
:101D80008FFEE4CE90FEE7CE93FEE8CE94FEE5CE45
:101D900091FEE6CE92FEE9CE95FEEACE96FE1200C8
:101DA000D9CFE6FFDACFE6FFE1CFD9FFE2CFDAFF06
:101DB000E652E65295CE33F096CE34F09EEC3CF0EF
:101DC00032C000F033C001F034C002F035C003F07F
:101DD000376A386A200E396E410E3A6E00C032F012
:101DE00001C033F002C034F003C035F063EC3DF0C5
:101DF00032C0B9FE33C0BAFE34C0BBFE35C0BCFE33
:101E00000E01875188112FE0006A016A7A0E026E76
:101E1000440E036E87CE33F088CE34F09EEC3CF057
:101E200032C004F033C005F034C006F035C007F00E
:101E300004C037F005C038F006C039F007C03AF0EA
:101E400000C032F001C033F002C034F003C035F0FE
:101E500063EC3DF032C0C5FE33C0C6FE34C0C7FEE1
:101E600035C0C8FE05D00E01C56BC66BC76BC86B0D
:101E70000E0189518A1129E089CE33F08ACE34F0DF
:101E80009EEC3CF032C000F033C001F034C002F0F0
:101E900035C003F000C037F001C038F002C039F09F
:101EA00003C03AF0D7CE32F0D8CE33F0D9CE34F0EA
:101EB000DACE35F063EC3DF032C0C9FE33C0CAFE65
:101EC00034C0CBFE35C0CCFE05D00E01C96BCA6B49
:101ED000CB6BCC6B0E018B518C1129E08BCE33F088
:101EE0008CCE34F09EEC3CF032C000F033C001F0F8
:101EF00034C002F035C003F0D7CE37F0D8CE38F07A
:101F0000D9CE39F0DACE3AF000C032F001C033F069
:101F100002C034F003C035F063EC3DF032C0CDFEBA
:101F200033C0CEFE34C0CFFE35C0D0FE05D00E018A
:101F3000CD6BCE6BCF6BD06B8DCE33F08ECE34F0BD
:101F40009EEC3CF032C0D1FE33C0D2FE34C0D3FE92
:101F500035C0D4FE670E006E5F0E016E026A00C0CF
:101F6000E6FF01C0E6FF7AEC04F0E552E552C5CE8B
:101F7000E6FFC6CEE6FFC7CEE6FFC8CEE6FF740E8C
:101F8000E66E000EE66E74EC3BF0F56E060EE15C5C
:101F900002E2E16AE552E16EF550610E006E5F0EFD
:101FA000016E026A00C0E6FF01C0E6FF7AEC04F0B1
:101FB000E552E552C9CEE6FFCACEE6FFCBCEE6FF3C
:101FC000CCCEE6FF740EE66E000EE66E74EC3BF0CF
:101FD000F56E060EE15C02E2E16AE552E16EF55053
:101FE0005B0E006E5F0E016E026A00C0E6FF01C06C
:101FF000E6FF7AEC04F0E552E552CDCEE6FFCECE18
:10200000E6FFCFCEE6FFD0CEE6FF740EE66E000E02
:10201000E66E74EC3BF0F56E060EE15C02E2E16AFE
:10202000E552E16EF550540E006E5F0E016E026ACD
:1020300000C0E6FF01C0E6FF7AEC04F0E552E5528D
:10204000D1CEE6FFD2CEE6FFD3CEE6FFD4CEE6FF7A
:10205000740EE66E000EE66E74EC3BF0F56E060E46
:10206000E15C02E2E16AE552E16EF550E552E552CB
:10207000E552E5CFDAFFE7CFD9FF1200D9CFE6FF6F
:10208000DACFE6FFE1CFD9FFE2CFDAFF060EE12497
:1020900002E3E168E652E16E040EDB6A050EDB6ADC
:1020A000330E006E5F0E016E026A00C0E6FF01C0D3
:1020B000E6FF7AEC04F0E552E552120EE66EE66AAF
:1020C000870EE66E0E0EE66E400EE66EE66A9FEC3A
:1020D0004AF0F56E060EE15C02E2E16AE552E16E5D
:1020E000F550000EE66EE66A100EE66EE66A870EA2
:1020F000E66E0E0EE66E13EC4DF0F56E060EE15C2C
:1021000002E2E16AE552E16EF550F3CFD5FEF4CF7D
:10211000D6FE870EDE6E0E0EDD6E020EDB6A030E3D
:10212000DB6A020EDBCF00F0030EDBCF01F0120EF4
:10213000005C000E015838E2DFCFE9FFDF2A010E14
:10214000DBCFEAFF01E3DB2AEF50E66EE66A020E20
:10215000DBCFE6FF030EDBCFE6FF1A0E006E5F0E4D
:10216000016E026A00C0E6FF01C0E6FF02C0E6FFA2
:10217000740EE66E000EE66E0FEC4EF0F56E090E74
:10218000E15C02E2E16AE552E16EF550740EE66E42
:10219000000EE66E53EC04F0E552E552020EDB2A27
:1021A000030E01E3DB2ABDD7D5CEE6FFD6CEE6FF90
:1021B0000C0E006E5F0E016E026A00C0E6FF01C0E9
:1021C000E6FF02C0E6FF740EE66E000EE66E0FEC50
:1021D0004EF0F56E070EE15C02E2E16AE552E16E57
:1021E000F550740EE66E000EE66E53EC04F0E55208
:1021F000E5520E0197510E01D51904E10E019851D7
:102200000E01D61901E1E3D0F80E006E5E0E016EEC
:10221000026A00C0E6FF01C0E6FF7AEC04F0E55276
:10222000E552D80E006E5E0E016E026A00C0E6FF37
:1022300001C0E6FF7AEC04F0E552E552120EE66EBC
:10224000E66A870EE66E0E0EE66E600EE66EE66AD3
:102250009FEC4AF0F56E060EE15C02E2E16AE5529F
:10226000E16EF550000EE66EE66A100EE66EE66A66
:10227000870EE66E0E0EE66E13EC4DF0F56E060E52
:10228000E15C02E2E16AE552E16EF550F3CFD5FE82
:10229000F4CFD6FE870EDE6E0E0EDD6E020EDB6A0A
:1022A000030EDB6A020EDBCF00F0030EDBCF01F082
:1022B000120E005C000E015838E2DFCFE9FFDF2A82
:1022C000010EDBCFEAFF01E3DB2AEF50E66EE66AA0
:1022D000020EDBCFE6FF030EDBCFE6FF1A0E006E29
:1022E0005F0E016E026A00C0E6FF01C0E6FF02C099
:1022F000E6FF740EE66E000EE66E0FEC4EF0F56E25
:10230000090EE15C02E2E16AE552E16EF550740EFD
:10231000E66E000EE66E53EC04F0E552E552020E56
:10232000DB2A030E01E3DB2ABDD7D5CEE6FFD6CEEE
:10233000E6FF0C0E006E5F0E016E026A00C0E6FF43
:1023400001C0E6FF02C0E6FF740EE66E000EE66E08
:102350000FEC4EF0F56E070EE15C02E2E16AE55229
:10236000E16EF550740EE66E000EE66E53EC04F06E
:10237000E552E5520E0197510E01D51904E10E0107
:1023800098510E01D6190EE0F80E006E5E0E016E29
:10239000026A00C0E6FF01C0E6FF7AEC04F0E552F5
:1023A000E55214D0C40E006E5E0E016E026A00C0CB
:1023B000E6FF01C0E6FF7AEC04F0E552E552020EBA
:1023C000F36E040EF3CFDBFF050EDB6A14D0C40EF0
:1023D000006E5E0E016E026A00C0E6FF01C0E6FFFD
:1023E0007AEC04F0E552E552010EF36E040EF3CFE1
:1023F000DBFF050EDB6A040EDBCF00F0050EDBCF42
:1024000001F000C0F3FF01C0F4FF00D0F56E060E2E
:10241000E15C02E2E16AE552E16EF550E552E5CF9A
:10242000DAFFE7CFD9FF1200D9CFE6FFDACFE6FF18
:10243000E1CFD9FFE2CFDAFFE652E652E652E652AA
:10244000B00E006E5E0E016E026A00C0E6FF01C0B3
:10245000E6FF7AEC04F0E552E552000EE66EE66A1D
:10246000100EE66EE66A870EE66E0E0EE66E13EC52
:102470004DF0F56E060EE15C02E2E16AE552E16EB6
:10248000F550F3CF97FEF4CF98FE870EDE6E0E0E5A
:10249000DD6E020EDB6A030EDB6A020EDBCF00F09C
:1024A000030EDBCF01F0120E005C000E015838E283
:1024B000DFCFE9FFDF2A010EDBCFEAFF01E3DB2AF2
:1024C000EF50E66EE66A020EDBCFE6FF030EDBCFCF
:1024D000E6FF1A0E006E5F0E016E026A00C0E6FF94
:1024E00001C0E6FF02C0E6FF740EE66E000EE66E67
:1024F0000FEC4EF0F56E090EE15C02E2E16AE55286
:10250000E16EF550740EE66E000EE66E53EC04F0CC
:10251000E552E552020EDB2A030E01E3DB2ABDD7AA
:1025200097CEE6FF98CEE6FF0C0E006E5F0E016EB2
:10253000026A00C0E6FF01C0E6FF02C0E6FF740EBB
:10254000E66E000EE66E0FEC4EF0F56E070EE15CE7
:1025500002E2E16AE552E16EF550740EE66E000E9D
:10256000E66E53EC04F0E552E552120EE66EE66AB2
:10257000870EE66E0E0EE66E400EE66EE66A17EC0D
:102580004BF0F56E060EE15C02E2E16AE552E16EA7
:10259000F550120EE66EE66A870EE66E0E0EE66ED9
:1025A000600EE66EE66A17EC4BF0F56E060EE15C27
:1025B00002E2E16AE552E16EF550010EF36EF46A53
:1025C00000D0F56E040EE15C02E2E16AE552E16ED4
:1025D000F550E552E5CFDAFFE7CFD9FF1200B9CECB
:1025E00037F0BACE38F0BBCE39F0BCCE3AF0BDCE23
:1025F00032F0BECE33F0BFCE34F0C0CE35F0CCECEE
:102600003CF032C0A5FE33C0A6FE34C0A7FE35C0E4
:10261000A8FEC5CE37F0C6CE38F0C7CE39F0C8CE4A
:102620003AF0A5CE32F0A6CE33F0A7CE34F0A8CE45
:1026300035F0B6EC3DF032C099FE33C09AFE34C09E
:102640009BFE35C09CFEA9CE37F0AACE38F0ABCEAB
:1026500039F0ACCE3AF0A5CE32F0A6CE33F0A7CE0C
:1026600034F0A8CE35F0CCEC3CF032C0B1FE33C033
:10267000B2FE34C0B3FE35C0B4FE376A386AA00E6D
:10268000396EC00E3A6EADCE32F0AECE33F0AFCE74
:1026900034F0B0CE35F028EC3FF0010A2DE1376A76
:1026A000386AC80E396E420E3A6EADCE32F0AECEFA
:1026B00033F0AFCE34F0B0CE35F031EC3FF0010A5C
:1026C0001BE1A5CE37F0A6CE38F0A7CE39F0A8CEC4
:1026D0003AF0B5CE32F0B6CE33F0B7CE34F0B8CE55
:1026E00035F0CDEC3CF032C0B5FE33C0B6FE34C0A0
:1026F000B7FE35C0B8FE05D00E01B56BB66BB76B33
:10270000B86BC9CE37F0CACE38F0CBCE39F0CCCECC
:102710003AF0B5CE32F0B6CE33F0B7CE34F0B8CE14
:1027200035F0B6EC3DF032C09DFE33C09EFE34C0A5
:102730009FFE35C0A0FEA5CEA9FEA6CEAAFEA7CEBE
:10274000ABFEA8CEACFECDCE37F0CECE38F0CFCE9D
:1027500039F0D0CE3AF0B1CE32F0B2CE33F0B3CEC3
:1027600034F0B4CE35F0B6EC3DF032C0A1FE33C04B
:10277000A2FE34C0A3FE35C0A4FE9DCE37F09ECE8F
:1027800038F09FCE39F0A0CE3AF099CE32F09ACE02
:1027900033F09BCE34F09CCE35F0CDEC3CF032C023
:1027A00000F033C001F034C002F035C003F0A1CE18
:1027B00037F0A2CE38F0A3CE39F0A4CE3AF000C064
:1027C00032F001C033F002C034F003C035F0CDEC7C
:1027D0003CF032C0C1FE33C0C2FE34C0C3FE35C0BF
:1027E000C4FEC1CEADFEC2CEAEFEC3CEAFFEC4CEE1
:1027F000B0FE376A386AC80E396E420E3A6EC1CEE4
:1028000032F0C2CE33F0C3CE34F0C4CE35F028EC73
:102810003FF0010A07E10E01C16BC26BC80EC36F26
:10282000420EC46F376A386A396A3A6AC1CE32F0EA
:10283000C2CE33F0C3CE34F0C4CE35F031EC3FF02D
:10284000010A05E10E01C16BC26BC36BC46B1200C0
:10285000D9CFE6FFDACFE6FFE1CFD9FFE2CFDAFF4B
:10286000E652E652A60E006E5E0E016E026A00C0CF
:10287000E6FF01C0E6FF7AEC04F0E552E5526CA2F7
:10288000FED7B9CEE6FFBACEE6FFBBCEE6FFBCCEA2
:10289000E6FF740EE66E000EE66E74EC3BF0F56E2D
:1028A000060EE15C02E2E16AE552E16EF5506CA2CF
:1028B000FED79E0E006E5E0E016E026A00C0E6FF3D
:1028C00001C0E6FF7AEC04F0E552E5526CA2FED7B7
:1028D000BDCEE6FFBECEE6FFBFCEE6FFC0CEE6FF32
:1028E000740EE66E000EE66E74EC3BF0F56E060EAE
:1028F000E15C02E2E16AE552E16EF5506CA2FED7BE
:10290000950E006E5E0E016E026A00C0E6FF01C009
:10291000E6FF7AEC04F0E552E5526CA2FED7C1CE98
:10292000E6FFC2CEE6FFC3CEE6FFC4CEE6FF740EDE
:10293000E66E000EE66E74EC3BF0F56E060EE15CA2
:1029400002E2E16AE552E16EF5506CA2FED78B0E11
:10295000006E5E0E016E026A00C0E6FF01C0E6FF77
:102960007AEC04F0E552E5526CA2FED737C2E6FFDE
:1029700038C2E6FF39C2E6FF3AC2E6FF740EE66EE1
:10298000000EE66E74EC3BF0F56E060EE15C02E2C2
:10299000E16AE552E16EF5506CA2FED7E552E552D0
:1029A000E552E5CFDAFFE7CFD9FF120014EC1AF0B9
:1029B000FB0EDBCFF3FFDB06F35000090AE062EC0D
:1029C0001AF0FA0ECDEC1AF0F3E1011CF1E1010E60
:1029D00001D0000E43EF1AF014EC1AF03B0EE12484
:1029E00002E3E168E652E16E010EDB6A020EDB6A89
:1029F000F90EDBCFF6FFFA0EDBCFF7FFFB0EDBCFD6
:102A0000F8FF0800F550DF6EDF5002E165EF19F0C6
:102A1000250EDF5C02E058EF19F0030EDB6A040EAE
:102A2000DB6A050EDB6A060EDB6A070EDB6A7CECEE
:102A300019F02D0EDF5C0CE02B0EDF5C09E0200EA0
:102A4000DF5C06E0230EDF5C03E0300EDF5C1AE1A2
:102A5000DF50300A14E0130A0FE0030A0AE00B0A01
:102A600005E0060AE4E1030EDB80E1D7030EDB821A
:102A7000DED7030EDB84DBD7030EDB86D8D7030E4D
:102A8000DB88D5D72A0EDF5C1BE178EC19F0C6ECA9
:102A900019F010E0030EDB8033683468130EDBCFCF
:102AA00038F0140EDBCF39F049EC3EF0040E31C0A3
:102AB000DBFF03D0130EAFEC19F07CEC19F00BD058
:102AC000090EDB6A1DEC1AF003E091EC1AF0FAD75C
:102AD000090EAFEC19F0030EDBB0DB982E0EDF5CB5
:102AE0001BE17CEC19F02A0EDF5C0BE178EC19F0AD
:102AF000C6EC19F003E1130E01EC1AF07CEC19F0AE
:102B00000BD0090EDB6A1DEC1AF003E091EC1AF011
:102B1000FAD7090E01EC1AF0680EDF5C07E17CECD5
:102B200019F0680EDF5C1DE1030E18D0740EDF5C37
:102B300017E07A0EDF5C14E0480EDF5C06E0540E0E
:102B4000DF5C03E05A0EDF5C02E1020E07D06C0E80
:102B5000DF5C03E06A0EDF5C04E1010E54EC1AF066
:102B6000CBDBDF506E0A01E17FD31E0A01E192D177
:102B7000200A01E18FD13F0A01E149D11A0A01E19E
:102B800046D10D0A01E143D1200A01E140D13A0AC0
:102B900001E13DD1200A01E13AD1260A01E135D116
:102BA0000D0A01E132D11A0A01E1D9D0200A4AE026
:102BB000300A1FE0460A0EE0250A01E083D3D9500F
:102BC000F90FE96EFF0EDA20EA6E010EEE5E000EDE
:102BD000EE5AEE5A62EC1AF0250EE66E97DB03E130
:102BE000011C01E169D35EEC1AF001E26BD3DB2A30
:102BF00069D3080EDB6A040EDB50010806E2040EFE
:102C0000DB0426EC1AF0DB508DDB080EDB5009E00C
:102C1000030EDB50010B05E174DB01E04DD3080E20
:102C2000DB6A66DBEFCFDFFFD6EC1AF003E1011CB5
:102C300001E142D35EEC1AF001E3DB2A62DB01E141
:102C400041D33AD3070EDB5002080FE1A2EC1AF091
:102C5000030E69EC1AF00E0EEECFDBFF0F0EEECF77
:102C6000DBFF100EEECFDBFF20D0F70EDBCF03F043
:102C7000F80EDBCF04F0020E035E000E045AF70ECE
:102C800003C0DBFFF80E04C0DBFF03C0E9FF04C094
:102C9000EAFF59EC1AF0026A0E0E00C0DBFF0F0EBD
:102CA00001C0DBFF100E02C0DBFF0E0EDBCFE6FF24
:102CB0000F0EDBCFE6FF100EDBCFE6FF3EEC4FF052
:102CC000E552E552E552130E32C0DBFF140E33C05D
:102CD000DBFF060EDB5005E0130E9DEC1AF001E25F
:102CE0006CDBC1EC1AF002E2130E39DB84EC1AF053
:102CF00006E0040E9DEC1AF002E2050E30DB030E36
:102D0000DBB005D0FEDA01E0D7D2080EDB6A090E8F
:102D1000DB6A0E0EDBCFF6FF0F0EDBCFF7FF100ED8
:102D2000DBCFF8FF0800F550DF6EDF5014E0C7EC92
:102D30001AF011E2D6EC1AF003E1011C01E1BCD259
:102D4000BDDB01E3DB2A090EDB2AD9500E0FE96E49
:102D5000000ECDDBE7D7D5DA01E1B4D2ADD2C8DAC7
:102D6000110EEECFDBFF120EEDCFDBFF110EDBCF2E
:102D7000E6FF120EDBCFE6FF30EC4FF0E552E552F6
:102D8000130EF3CFDBFF140EF4CFDBFF060EDB5088
:102D900004E0130ED2DB01E210DBC1EC1AF002E218
:102DA000130EDDDAB1DB05E0040EC7DB02E2050E2F
:102DB000D6DA030EDBB005D0A4DA01E07DD2080E2E
:102DC000DB6A090EDB6A110EDBCFE9FF120EDBCFE7
:102DD000EAFFEFCFDFFFDF5014E0D9DB12E2E6DBE2
:102DE00003E1011C01E168D269DB01E3DB2A090E82
:102DF000DB2A110EDB2ADBCFE9FF120EE8E3DB2A28
:102E0000E6D77FDA01E15ED257D2030EDB8E070EE2
:102E1000DB0410E197DB040E5CDB0A0EEECFDBFF78
:102E20000B0EEECFDBFF0C0EEECFDBFF0D0EEECF69
:102E3000DBFF6CD0070EDB5003082CE1030EDBAE8A
:102E40000DD0B4DA020E78DAEFCF00F0016A026A30
:102E5000036A00AE39D00168026835D0F70EDBCFC7
:102E600001F0F80EDBCF02F0020E015E000E025AF6
:102E7000F70E01C0DBFFF80E02C0DBFF01C0E9FF67
:102E800002C0EAFFEFCF00F00A0E00C0DBFF0B0E1E
:102E9000DB6A38D0070EDB50020809E1030EDBAE17
:102EA00004D05BDB02AE10D00ED057DB0DD0030E8A
:102EB000DBAE12D07BDA020E3FDAFBDA026A036A7B
:102EC00001AE02D002680368E4DA0C0E02C0DBFF38
:102ED0000D0E03C0DBFF1AD0F70EDBCF02F0F80EA9
:102EE000DBCF03F0020E025E000E035AF70E02C0A3
:102EF000DBFFF80E03C0DBFF02C0E9FF03C0EAFFFF
:102F0000D8DAC7DA0C0EDB6A0D0EDB6A060EDB5070
:102F100005E1010EF36E050EF3CFDBFF150EDB6A44
:102F2000160EDB6AD950370F006E000EDA20016EE4
:102F3000390E00C0DBFF3A0E01C0DBFF380EDB6A42
:102F4000080EDB6A0A0EB0DADF50780A12E0200AB7
:102F500010E0280A0CE0200A0AE03F0A06E00D0A09
:102F600002E0200A08E1020E05D0080E03D0080E88
:102F7000DF26100E99DA030EDBBE02D0DB92DB9463
:102F8000DB50800B24E08CDAD890030EEB50000A63
:102F900008E6000EEE5C000EEE58000EEE58000E35
:102FA000EE5815E215DA3668376838683968F8EC93
:102FB0004EF00A0E2DC0DBFF0B0E2EC0DBFF0C0EF9
:102FC0002FC0DBFF0D0E30C0DBFF2D0E08D0030E2F
:102FD000DBA202D02B0E03D0DBA408D0200EF36EB0
:102FE000170EF3CFDBFF150EDB2A02D0170EDB6ABC
:102FF000050EDB5003E1B9D901E189D00E0E006E58
:10300000A40E016E000E026E070EDBCF03F0046A01
:10301000056A066A03C036F004C037F005C038F010
:1030200006C039F0D5D98BEC50F000502D24F36E4A
:1030300001502E20F46E02502F20F86EF4CFF7FFCF
:10304000F3CFF6FF0800090EF5CFDBFF580EDF5C6B
:103050000FE1610EF36E090E7DD90AE3200E006EBA
:10306000090EDBCFE7FF0050E75E090EE7CFDBFF7D
:10307000070EDBCF00F0016A026A036A11DA00C0B2
:1030800036F001C037F002C038F003C039F0EECF9F
:1030900031F0EECF32F0EECF33F0EFCF34F08BECF7
:1030A00050F034C0EDFF33C0EDFF32C0EDFF31C052
:1030B000EFFF390EDBCFE9FFDB063A0EDBCFEAFF8D
:1030C00001E2DB06090EDBCFEFFF150EDB2A4DD93F
:1030D00095E1030EDBA61DD06F0EDF5C06E1C3D9C0
:1030E00018E3150EDB285DDA14D0780EDF5C09E0FA
:1030F000580EDF5C06E0620EDF5C03E0420EDF5C30
:1031000008E1020EF36E160EF3CFDBFF02D0150EB0
:10311000DB6A030EDB50100B0EE0040EDBCF00F079
:10312000050EDB50D880005406E2060EDB5003E1AA
:10313000040EDB5036DA97D90AE2050EDBCFE7FF43
:10314000150EDB50E75E050EE7CFDBFF02D0050E64
:10315000DB6A040EDBCF00F0160E47D9D88000548E
:1031600014E2160EDBCFE6FF150EDBCFE6FF040EF2
:10317000DBCFE6FF050EDB50E552E75CE552D88079
:10318000E754E552D880E75461D9030EDB50010BB8
:103190000BE1080EDB5008E0B4D801E08DD0080E3A
:1031A000DB50C0D8080EDB6A170EDB5007E08AD967
:1031B000170EF3D903E1011C01E17ED0160EDB509E
:1031C00016E080D9300EE66EA1D802E1011C74E051
:1031D00079D9DFCFE6FFB6EC4EF0E552E552E55285
:1031E000F4CF01F00001F31C02E1011C65E0050EC3
:1031F000DBCF00F0160EDB50D880005409E2050E3C
:10320000DBCFE7FF160EDB50E75E050EE7CFDBFFF7
:10321000300EE66E050ECDD94FE1390EDB2ADBCF3D
:10322000E9FF3A0E01E3DB2ADBCFEAFF090EEFCF1D
:10323000DBFFDB500EE046D9090EAFD902E1011CDD
:103240003BE0390EDB2ADBCFE9FF3A0EEDE3DB2A68
:10325000EBD757D831E1160EDBCFE6FF080EC5D805
:10326000E552E7245FD82ED0070EDB50030A1CE09E
:10327000010A14E0030A07E07DD9DBCFEEFF020E5E
:10328000DBCFEDFF1FD0F7D8056A03AE02D004688C
:1032900005682ED8BED805C0EEFF14D0ECD803BE0A
:1032A000046826D8B6D80ED065D9DBCFEFFF0AD098
:1032B0007DD905E1011C03E1F368F46810D0FED864
:1032C00001E3DB2A7BD901EF15F0010EDBCF00F023
:1032D000020EDBCF01F000C0F3FF01C0F4FFF56E7A
:1032E0003B0EE15C02E2E16AE552E16EF550CBD0C3
:1032F00029D9020E69EF1AF061D90800F550DF6E86
:103300001200200EE66E080ED9EF1AF0B6EC4EF061
:10331000E552E552E552F3CF00F0F4CF01F00001A1
:10332000F31C1200006E016AD950010F4DD90050F4
:10333000EE260150ED221200045E000E055AF70E33
:1033400004C0DBFFF80E05C0DBFF04C0E9FF05C0C9
:10335000EAFF1200DBCFF4FFF350F45C1200DB5005
:10336000E76E040EE7CFDBFF12000A0EDBCF00F0A2
:103370000B0EDBCF01F00C0EDBCF02F00D0EDBCF1E
:1033800003F000500110021003101200130EEECFD4
:10339000DBFF140EEDCFDBFF130EDBCF00F0140EBE
:1033A000DBCF01F00001800E01141200F70EDBCF1D
:1033B00004F0F80EDBCF05F01200050EDB50E66ED0
:1033C000D950130F01D9E552E750EE6EED6A1200A5
:1033D0000A0EDBCF31F00B0EDBCF32F00C0EDBCF61
:1033E00033F00D0EDBCF34F01200DBCFE6FF150E0D
:1033F000DBCFE6FF050EDB50E552E724E552E7247C
:103400001200DB50CED8010EF36E060EF3CFDBFFB9
:103410001200EE50EFCFEAFFE96E02C0EEFF03C0EC
:10342000EEFF04C0EEFF1200D9CFE6FFDACFE6FFD1
:10343000E1CFD9FFE2CFDAFF1200DFCFE6FFE66A85
:10344000CBEC51F0E552E552F3501200E76E080E56
:10345000E7CFDBFF1200EECF00F0EECF01F0EFCFB1
:1034600002F0036A1200050EDBCF00F0150EDB50F0
:10347000D88000541200010EDBCF02F0020EDBCF29
:1034800003F0046A1200E552E5CFDAFFE7CFD9FF77
:1034900012000A0E00C0DBFF0B0E01C0DBFF1200A2
:1034A000D9500A0FE4EF1AF0F36E070EF3CFDBFFEB
:1034B0001200EECF00F0EFCF01F01200010EDB2A78
:1034C000020E1200FC0EDBCFE6FFFD0EDBCFE6FFA7
:1034D0001200005E000E015AF70E00C0DBFFF80E6E
:1034E00001C0DBFF00C0E9FF01C0EAFF1200DA20E3
:1034F000EA6EEF2AEECFF6FF000EEF22EECFF7FFD7
:10350000EF22EECFF8FF1200040EDBCFE6FF130E22
:10351000DB50E552E75C9ADFDB5004DF060EDB5040
:103520001200090EDB500A0DF350DF24D00FE76EB6
:10353000090EE7CFDBFF7CEF19F0DB50F36E050ED1
:10354000AAEF19F0F70EDBCF00F0F80EDBCF01F099
:103550001200DFCFE6FF86EF19F028DF030EECDE66
:103560002BEF1AF0D6EC14F0E552E552E552E55295
:1035700000091200BDDEEE50EFCFEAFFE96E010E4A
:103580001200130EDB50F36E040EAAEF19F0040EB6
:10359000DB50F36E090EAAEF19F0DBCFE6FF86EFE2
:1035A00019F0E76E050EE7CFDBFF12008BDFA9EF06
:1035B0001AF0DBCFE6FF86DFB2EF1AF0D950F90F31
:1035C000E96EFF0E77EF1AF0E96E000EDA20EA6E70
:1035D0001200D9CFE6FFDACFE6FFE1CFD9FFE2CF85
:1035E000DAFFE652850E006E5D0E016E026A00C0C3
:1035F000E6FF01C0E6FF7AEC04F0E552E552000177
:103600006C6B6D6B6E6B6F6B0001686B696B6A6BDB
:103610006B6BDF6A080EDF5C0BE21EDBF3CF00F0A2
:10362000F4CF01F00050011001E1F7D7DF2AF2D703
:1036300009D845EC1FF0E552E552E5CFDAFFE7CFB8
:10364000D9FF1200D9CFE6FFDACFE6FFE1CFD9FFED
:10365000E2CFDAFF0C0EE12402E3E168E652E16E0C
:10366000086A096A800E0A6E490E0B6E37C237F07F
:1036700038C238F039C239F03AC23AF008C032F0F4
:1036800009C033F00AC034F00BC035F0B6EC3DF0A1
:1036900032C004F033C005F034C006F035C007F086
:1036A000106A116A800E126E490E136E68C031F0F6
:1036B00069C032F06AC033F06BC034F0B3EC3CF058
:1036C00032C014F033C015F034C016F035C017F016
:1036D00014C037F015C038F016C039F017C03AF0F2
:1036E00010C032F011C033F012C034F013C035F006
:1036F000CCEC3CF032C00CF033C00DF034C00EF016
:1037000035C00FF00CC037F00DC038F00EC039F0E6
:103710000FC03AF004C032F005C033F006C034F0F8
:1037200007C035F063EC3DF032C000F033C001F06B
:1037300034C002F035C003F037C237F038C238F079
:1037400039C239F03AC23AF000C032F001C033F069
:1037500002C034F003C035F0CCEC3CF0080E32C0AF
:10376000DBFF090E33C0DBFF0A0E34C0DBFF0B0E9C
:1037700035C0DBFFD950080FE96E000EDA20EA6E83
:10378000EECFE6FFEECFE6FFEECFE6FFEFCFE6FFB0
:103790003AEC26F0E552E552E552E55231C06CF0C4
:1037A00032C06DF033C06EF034C06FF00E01935133
:1037B000941160E0046A056A800E066E3F0E076E83
:1037C00093CE33F094CE34F09EEC3CF032C00CF04B
:1037D00033C00DF034C00EF035C00FF0376A386AD0
:1037E000C80E396E420E3A6E0CC032F00DC033F086
:1037F0000EC034F00FC035F063EC3DF032C008F07D
:1038000033C009F034C00AF035C00BF008C037F0FF
:1038100009C038F00AC039F00BC03AF004C032F0E9
:1038200005C033F006C034F007C035F0CDEC3CF0F5
:1038300032C000F033C001F034C002F035C003F0F4
:1038400000C037F001C038F002C039F003C03AF0D0
:103850006CC032F06DC033F06EC034F06FC035F024
:10386000B6EC3DF032C06CF033C06DF034C06EF099
:1038700035C06FF00E019151921160E0046A056A43
:103880008C0E066E420E076E91CE33F092CE34F05F
:103890009EEC3CF032C00CF033C00DF034C00EF0A2
:1038A00035C00FF0376A386AC80E396E420E3A6E6C
:1038B0000CC032F00DC033F00EC034F00FC035F044
:1038C00063EC3DF032C008F033C009F034C00AF0B8
:1038D00035C00BF008C037F009C038F00AC039F025
:1038E0000BC03AF004C032F005C033F006C034F02B
:1038F00007C035F0B6EC3DF032C000F033C001F047
:1039000034C002F035C003F000C037F001C038F019
:1039100002C039F003C03AF06CC032F06DC033F031
:103920006EC034F06FC035F0CDEC3CF032C06CF0BE
:1039300033C06DF034C06EF035C06FF00E018F51A2
:10394000901101E10DD1046A056A8C0E066E420EDB
:10395000076ED7CE37F0D8CE38F0D9CE39F0DACEE0
:103960003AF004C032F005C033F006C034F007C0AE
:1039700035F0B6EC3DF032C000F033C001F034C099
:1039800002F035C003F08FCE33F090CE34F09EECD1
:103990003CF032C008F033C009F034C00AF035C042
:1039A0000BF008C037F009C038F00AC039F00BC07E
:1039B0003AF000C032F001C033F002C034F003C06E
:1039C00035F063EC3DF032C0DEFF33C0DEFF34C0C3
:1039D000DEFF35C0DDFFDD52DD52EFCE37F0F0CE39
:1039E00038F0F1CE39F0F2CE3AF06CC032F06DC062
:1039F00033F06EC034F06FC035F0CCEC3CF0040E08
:103A000032C0DBFF050E33C0DBFF060E34C0DBFF28
:103A1000070E35C0DBFF040EDBCF00F0050EDBCF59
:103A200001F0060EDBCF02F0070EDBCF03F0D9CF9B
:103A3000E9FFDACFEAFFEECF04F0EECF05F0EECFEC
:103A400006F0EFCF07F004C037F005C038F006C02D
:103A500039F007C03AF000C032F001C033F002C0C4
:103A600034F003C035F028EC3FF0010A27E1D9CF4C
:103A7000E9FFDACFEAFFEECF00F0EECF01F0EECFB4
:103A800002F0EFCF03F000C037F001C038F002C001
:103A900039F003C03AF0EFCE32F0F0CE33F0F1CE91
:103AA00034F0F2CE35F0CDEC3CF032C06CF033C0E7
:103AB0006DF034C06EF035C06FF052D0040EDBCF25
:103AC00000F0050EDBCF01F0060EDBCF02F0070E93
:103AD000DBCF03F0D9CFE9FFDACFEAFFEECF04F076
:103AE000EECF05F0EECF06F0EFCF07F004C037F0D1
:103AF00005C038F006C039F007C03AF000C032F017
:103B000001C033F002C034F003C035F031EC3FF0B7
:103B1000010A26E1D9CFE9FFDACFEAFFEECF00F0C4
:103B2000EECF01F0EECF02F0EFCF03F000C037F0A0
:103B300001C038F002C039F003C03AF0EFCE32F0E5
:103B4000F0CE33F0F1CE34F0F2CE35F0CCEC3CF0E8
:103B500032C06CF033C06DF034C06EF035C06FF021
:103B60006C0EE66E000EE66E10D8E552E552F56E6C
:103B70000C0EE15C02E2E16AE552E16EF550E552BD
:103B8000E5CFDAFFE7CFD9FF1200D9CFE6FFDACFD2
:103B9000E6FFE1CFD9FFE2CFDAFFFC0EDBCFE9FF92
:103BA000FD0EDBCFEAFFEECF00F0EECF01F0EECF5F
:103BB00002F0EFCF03F0376A386A480E396E420ED2
:103BC0003A6E00C032F001C033F002C034F003C0DE
:103BD00035F031EC3FF0010A0DE0FC0EDBCFE9FFE0
:103BE000FD0EDBCFEAFFEE6AEE6A480EEE6E420E85
:103BF000EE6E2CD0FC0EDBCFE9FFFD0EDBCFEAFF33
:103C0000EECF00F0EECF01F0EECF02F0EFCF03F0F9
:103C1000376A386AA00E396EC10E3A6E00C032F0B3
:103C200001C033F002C034F003C035F028EC3FF09F
:103C3000010A0CE0FC0EDBCFE9FFFD0EDBCFEAFF53
:103C4000EE6AEE6AA00EEE6EC10EEE6EE552E5CFA4
:103C5000DAFFE7CFD9FF1200D9CFE6FFDACFE6FFD0
:103C6000E1CFD9FFE2CFDAFF080EE12402E3E168F9
:103C7000E652E16EECD9F3CF00F0F4CF01F0010E83
:103C8000001801E1015055E160C0E6FF61C0E6FFA8
:103C900062C0E6FF63C0E6FF5DD8E552E552E5523B
:103CA000E55231C0DEFF32C0DEFF33C0DEFF34C07C
:103CB000DDFFDD52DD5264C0E6FF65C0E6FF66C091
:103CC000E6FF67C0E6FF46D8E552E552E552E55209
:103CD000040E31C0DBFF050E32C0DBFF060E33C021
:103CE000DBFF070E34C0DBFF040EDBCF00F0050E58
:103CF000DBCF01F0060EDBCF02F0070EDBCF03F0C7
:103D0000D9CFE9FFDACFEAFFEE5000240001686F57
:103D1000EE5001200001696FEE50022000016A6F31
:103D2000EE50032000016B6F010EF36EF46A04D0B5
:103D300003D0F36AF46A00D0F56E080EE15C02E28B
:103D4000E16AE552E16EF550E552E5CFDAFFE7CFE3
:103D5000D9FF1200D9CFE6FFDACFE6FFE1CFD9FFD6
:103D6000E2CFDAFFE652E652E652E652FB0EDBCF36
:103D700000F0016A026A036AFC0EDBCF04F0056AF8
:103D8000066A076A080E1F0B07E0D890043605364E
:103D900006360736E806F9E1045000120550011214
:103DA0000650021207500312D950FA0FE96EFF0EA7
:103DB000DA20EA6EEE52EE52EE52EF500F0B086E22
:103DC000096A0A6A0B6A100E1F0B07E0D8900836C2
:103DD00009360A360B36E806F9E108500012095098
:103DE00001120A5002120B50031200C0DFFF010E35
:103DF00001C0DBFF020E02C0DBFF030E03C0DBFFCE
:103E0000D950FA0FE96EFF0EDA20EA6EEE52EE524A
:103E1000EE52EF50100B20E0D950FA0FE96EFF0E72
:103E2000DA20EA6EEE52EE52EE52EF50200B0AE12B
:103E3000D9CFE9FFDACFEAFFEE52EE52F00EEE12E2
:103E4000EE680AD0D9CFE9FFDACFEAFFEE52EE52A0
:103E5000100EEE26000EEE22DECF31F0DECF32F075
:103E6000DECF33F0DDCF34F0DD52DD5200D0F56E21
:103E7000040EE15C02E2E16AE552E16EF550E552C2
:103E8000E5CFDAFFE7CFD9FF120068C0E6FF69C0CF
:103E9000E6FF6AC0E6FF6BC0E6FF690E006E5D0ECE
:103EA000016E026A00C0E6FF01C0E6FF02C0E6FF45
:103EB000740EE66E000EE66E0FEC4EF0F56E090E17
:103EC000E15C02E2E16AE552E16EF550740EE66EE5
:103ED000000EE66E53EC04F0E552E5526CC0E6FFCE
:103EE0006DC0E6FF6EC0E6FF6FC0E6FF740EE66EC3
:103EF000000EE66E74EC3BF0F56E060EE15C02E23D
:103F0000E16AE552E16EF5501200D9CFE6FFDACF53
:103F1000E6FFE1CFD9FFE2CFDAFFFA0EDBCFE6FF13
:103F2000E66AFB0EDBCFE6FFE66AFC0EDBCFE6FFC0
:103F3000E66AD950FA0FE96EFF0EDA20EA6EEE5209
:103F4000EE52EE52EF500F0BE66EE66AD950FA0FC2
:103F5000E96EFF0EDA20EA6EEE52EE52EE52EF50AC
:103F6000100B01E0010EE66EE66AD950FA0FE96E19
:103F7000FF0EDA20EA6EEE52EE52EE52EF50200BB8
:103F800001E0010EE66EE66AD950FA0FE96EFF0E07
:103F9000DA20EA6EEE52EE52EE52EF50400B01E0A4
:103FA000010EE66EE66AD950FA0FE96EFF0EDA20CE
:103FB000EA6EEE52EE52EE52EF50800B01E0010E2F
:103FC000E66EE66AFD0EDBCFE6FFE66AFC0EDBCFAF
:103FD000E6FFE66AFB0EDBCFE6FFE66AFA0EDBCF12
:103FE000E6FFE66AD950FA0FE96EFF0EDA20EA6EB4
:103FF000EECFE6FFEECFE6FFEECFE6FFEFCFE6FF38
:10400000BB0E006E5C0E016E026A00C0E6FF01C0CE
:10401000E6FF02C0E6FF740EE66E000EE66E0FECE1
:104020004EF0F56E210EE15C02E2E16AE552E16ECE
:10403000F550740EE66E000EE66E53EC04F0E55299
:10404000E552E552E5CFDAFFE7CFD9FF1200D9CF2D
:10405000E6FFDACFE6FFE1CFD9FFE2CFDAFF060EC7
:10406000E12402E3E168E652E16E040EDB6A050E2C
:10407000DB6ADE6ADE6ADE6ADD6ADD52DD5282906C
:10408000000082A803D0F368F46845D010EC52F029
:10409000E76E030EE7CFDBFF10EC52F0E76E020E87
:1040A000E7CFDBFF10EC52F0E76E010EE7CFDBFF4E
:1040B0008280D9CFE9FFDACFEAFFEE52EE52EE521C
:1040C000EF50800B28E1D9CFE9FFDACFEAFFEE52BB
:1040D000EE52EE52EF50400B10E0DFCF64F0010ED5
:1040E000DBCF65F0020EDBCF66F0030EDBCF67F0AF
:1040F000010EF36EF46A0FD00ED0DFCF60F0010E28
:10410000DBCF61F0020EDBCF62F0030EDBCF63F09A
:10411000F36AF46A00D0F56E060EE15C02E2E16A31
:10412000E552E16EF550E552E5CFDAFFE7CFD9FF72
:104130001200D9CFE6FFDACFE6FFE1CFD9FFE2CF19
:10414000DAFFE652E652E652E6523C0E006E5C0E94
:10415000016E026A00C0E6FF01C0E6FF7AEC04F0DF
:10416000E552E552230E006E5C0E016E026A00C03D
:10417000E6FF01C0E6FF7AEC04F0E552E5520D0ED1
:10418000006E5C0E016E026A00C0E6FF01C0E6FF31
:104190007AEC04F0E552E552F90E006E5B0E016E0A
:1041A000026A00C0E6FF01C0E6FF7AEC04F0E552C7
:1041B000E552E80E006E5B0E016E026A00C0E6FF7B
:1041C00001C0E6FF7AEC04F0E552E552D30E006E32
:1041D0005B0E016E026A00C0E6FF01C0E6FF7AECEA
:1041E00004F0E552E552C00E006E5B0E016E026AED
:1041F00000C0E6FF01C0E6FF7AEC04F0E552E552AC
:10420000AA0E006E5B0E016E026A00C0E6FF01C0DE
:10421000E6FF7AEC04F0E552E5529B0E006E5B0E71
:10422000016E026A00C0E6FF01C0E6FF7AEC04F00E
:10423000E552E552890E006E5B0E016E026A00C007
:10424000E6FF01C0E6FF7AEC04F0E552E5526A0EA3
:10425000006E5B0E016E026A00C0E6FF01C0E6FF61
:104260007AEC04F0E552E552A4AAFED7D0EC50F067
:10427000E76E010EE7CFDBFF010EDB50510A02E1D2
:1042800026EF26F0200A02E126EF26F03B0A02E1A3
:1042900011EF26F0200A02E111EF26F0230A02E1D5
:1042A000EEEF25F0200A02E1EEEF25F0210A02E10F
:1042B000E3EF25F0200A02E1E3EF25F02F0A02E107
:1042C000DEEF25F0200A02E1DEEF25F0210A02E10F
:1042D000DBEF25F0200A02E1DBEF25F0230A01E104
:1042E000F8D3200A01E1F5D3210A01E1D3D3200A52
:1042F00001E1D0D3270A01E1BED3200A01E1BBD3FB
:10430000210A01E11FD1200A01E11CD1230A04E0A6
:10431000200A02E029EF26F0DF6ADF5001E011D128
:104320004F0E006E5B0E016E026A00C0E6FF01C018
:10433000E6FF7AEC04F0E552E552350E006E5B0EB6
:10434000016E026A00C0E6FF01C0E6FF7AEC04F0ED
:10435000E552E5521C0E006E5B0E016E026A00C053
:10436000E6FF01C0E6FF7AEC04F0E552E552FF0EED
:10437000006E5A0E016E026A00C0E6FF01C0E6FF41
:104380007AEC04F0E552E552E60E006E5A0E016E2C
:10439000026A00C0E6FF01C0E6FF7AEC04F0E552D5
:1043A000E552DA0E006E5A0E016E026A00C0E6FF98
:1043B00001C0E6FF7AEC04F0E552E552A4AAFED76C
:1043C000D0EC50F0E76E010EE7CFDBFF010EDB50C3
:1043D000510A01E1B1D0200A01E1AED0140A01E195
:1043E0009CD0200A01E18AD0210A01E178D0200A7C
:1043F00067E0270A56E0200A45E0210A34E0200A57
:1044000023E0230A12E0200A01E099D0C90E006ED1
:104410005A0E016E026A00C0E6FF01C0E6FF7AECA8
:1044200004F0E552E55285948BD0B70E006E5A0E1B
:10443000016E026A00C0E6FF01C0E6FF7AEC04F0FC
:10444000E552E55285847CD0A60E006E5A0E016EB0
:10445000026A00C0E6FF01C0E6FF7AEC04F0E55214
:10446000E55285906DD0940E006E5A0E016E026A70
:1044700000C0E6FF01C0E6FF7AEC04F0E552E55229
:1044800085805ED0840E006E5A0E016E026A00C0F6
:10449000E6FF01C0E6FF7AEC04F0E552E5528592B2
:1044A0004FD0730E006E5A0E016E026A00C0E6FF16
:1044B00001C0E6FF7AEC04F0E552E552858240D077
:1044C0005F0E006E5A0E016E026A00C0E6FF01C068
:1044D000E6FF7AEC04F0E552E552859631D04A0EBB
:1044E000006E5A0E016E026A00C0E6FF01C0E6FFD0
:1044F0007AEC04F0E552E552858622D03A0E006E41
:104500005A0E016E026A00C0E6FF01C0E6FF7AECB7
:1045100004F0E552E552859A13D0290E006E5A0E2A
:10452000016E026A00C0E6FF01C0E6FF7AEC04F00B
:10453000E552E552858A04D0010EDF6E01D000D02D
:10454000ECD688D3DF6ADF5001E093D2120E006E02
:104550005A0E016E026A00C0E6FF01C0E6FF7AEC67
:1045600004F0E552E552FB0E006E590E016E026A30
:1045700000C0E6FF01C0E6FF7AEC04F0E552E55228
:10458000E20E006E590E016E026A00C0E6FF01C025
:10459000E6FF7AEC04F0E552E552CA0E006E590EC1
:1045A000016E026A00C0E6FF01C0E6FF7AEC04F08B
:1045B000E552E552B30E006E590E016E026A00C05C
:1045C000E6FF01C0E6FF7AEC04F0E552E5529A0EF0
:1045D000006E590E016E026A00C0E6FF01C0E6FFE0
:1045E0007AEC04F0E552E5528B0E006E590E016E26
:1045F000026A00C0E6FF01C0E6FF7AEC04F0E55273
:10460000E5527C0E006E590E016E026A00C0E6FF94
:1046100001C0E6FF7AEC04F0E552E552690E006E47
:10462000590E016E026A00C0E6FF01C0E6FF7AEC97
:1046300004F0E552E552530E006E590E016E026A07
:1046400000C0E6FF01C0E6FF7AEC04F0E552E55257
:10465000490E006E590E016E026A00C0E6FF01C0ED
:10466000E6FF7AEC04F0E552E552A4AAFED7D0ECBE
:1046700050F0E76E010EE7CFDBFF010EDB50510A71
:1046800001E1F2D1200A01E1EFD13B0A01E1C0D101
:10469000200A01E1BDD1230A01E18ED1200A01E106
:1046A0008BD1210A01E15CD1200A01E159D12F0A05
:1046B00001E12AD1200A01E127D1210A01E1F8D044
:1046C000200A01E1F5D0230A01E1C6D0200A01E168
:1046D000C3D0210A01E194D0200A01E191D0270A38
:1046E00063E0200A61E0210A33E0200A31E0230A76
:1046F00003E0200A01E0BBD1360E006E590E016EB8
:10470000026A00C0E6FF01C0E6FF7AEC04F0E55261
:10471000E5520E0112510EE02E0E006E590E016E82
:10472000026A00C0E6FF01C0E6FF7AEC04F0E55241
:10473000E5520DD0240E006E590E016E026A00C0C3
:10474000E6FF01C0E6FF7AEC04F0E552E55290D1B5
:10475000100E006E590E016E026A00C0E6FF01C025
:10476000E6FF7AEC04F0E552E5520E0118510EE036
:104770002E0E006E590E016E026A00C0E6FF01C0E7
:10478000E6FF7AEC04F0E552E5520DD0240E006EFF
:10479000590E016E026A00C0E6FF01C0E6FF7AEC26
:1047A00004F0E552E55264D1FA0E006E580E016E27
:1047B000026A00C0E6FF01C0E6FF7AEC04F0E552B1
:1047C000E5520E0124510EE02E0E006E590E016EC0
:1047D000026A00C0E6FF01C0E6FF7AEC04F0E55291
:1047E000E5520DD0240E006E590E016E026A00C013
:1047F000E6FF01C0E6FF7AEC04F0E552E55238D15D
:10480000E50E006E580E016E026A00C0E6FF01C0A0
:10481000E6FF7AEC04F0E552E5520E012A510EE073
:104820002E0E006E590E016E026A00C0E6FF01C036
:10483000E6FF7AEC04F0E552E5520DD0240E006E4E
:10484000590E016E026A00C0E6FF01C0E6FF7AEC75
:1048500004F0E552E5520CD1D10E006E580E016EF7
:10486000026A00C0E6FF01C0E6FF7AEC04F0E55200
:10487000E5520E011E510EE02E0E006E590E016E15
:10488000026A00C0E6FF01C0E6FF7AEC04F0E552E0
:10489000E5520DD0240E006E590E016E026A00C062
:1048A000E6FF01C0E6FF7AEC04F0E552E552E0D005
:1048B000BB0E006E580E016E026A00C0E6FF01C01A
:1048C000E6FF7AEC04F0E552E5520E0130510EE0BD
:1048D0002E0E006E590E016E026A00C0E6FF01C086
:1048E000E6FF7AEC04F0E552E5520DD0240E006E9E
:1048F000590E016E026A00C0E6FF01C0E6FF7AECC5
:1049000004F0E552E552B4D0AF0E006E580E016EC1
:10491000026A00C0E6FF01C0E6FF7AEC04F0E5524F
:10492000E5520E0136510EE02E0E006E590E016E4C
:10493000026A00C0E6FF01C0E6FF7AEC04F0E5522F
:10494000E5520DD0240E006E590E016E026A00C0B1
:10495000E6FF01C0E6FF7AEC04F0E552E55288D0AC
:10496000A30E006E580E016E026A00C0E6FF01C081
:10497000E6FF7AEC04F0E552E5520E013C510EE000
:104980002E0E006E590E016E026A00C0E6FF01C0D5
:10499000E6FF7AEC04F0E552E5520DD0240E006EED
:1049A000590E016E026A00C0E6FF01C0E6FF7AEC14
:1049B00004F0E552E5525CD0930E006E580E016E85
:1049C000026A00C0E6FF01C0E6FF7AEC04F0E5529F
:1049D000E5520E010C510EE02E0E006E590E016EC6
:1049E000026A00C0E6FF01C0E6FF7AEC04F0E5527F
:1049F000E5520DD0240E006E590E016E026A00C001
:104A0000E6FF01C0E6FF7AEC04F0E552E55230D053
:104A1000800E006E580E016E026A00C0E6FF01C0F3
:104A2000E6FF7AEC04F0E552E5520E0106510EE085
:104A30002E0E006E590E016E026A00C0E6FF01C024
:104A4000E6FF7AEC04F0E552E5520DD0240E006E3C
:104A5000590E016E026A00C0E6FF01C0E6FF7AEC63
:104A600004F0E552E55204D0010EDF6E01D000D013
:104A70006AD5DF6AEFD02CEC1EF0F3CF00F0F4CF54
:104A800001F00050011001E1F6D722EC1BF045ECDB
:104A90001FF0E0D0770E006E580E016E026A00C063
:104AA000E6FF01C0E6FF7AEC04F0E552E55294928D
:104AB000C80EE66E5DEC51F0E552C80EE66E5DEC98
:104AC00051F0E552C80EE66E5DEC51F0E55294826D
:104AD000C1D0420E006E580E016E026A00C0E6FFA1
:104AE00001C0E6FF7AEC04F0E552E552030EE66EF3
:104AF000740EE66E000EE66E2DEC50F0E552E552B7
:104B0000E552740EE66E000EE66E9AEC4DF0E5523C
:104B1000E552020EF3CFDBFF030EF4CFDBFF020EF4
:104B2000DBCFE6FF030EDBCFE6FF360E006E580E3E
:104B3000016E026A00C0E6FF01C0E6FF02C0E6FFA8
:104B4000740EE66E000EE66E0FEC4EF0F56E070E7C
:104B5000E15C02E2E16AE552E16EF550740EE66E48
:104B6000000EE66E53EC04F0E552E552D950020F08
:104B7000E96E000EDA20EA6E640ED880EE54000E64
:104B8000ED540EE22B0E006E580E016E026A00C04C
:104B9000E6FF01C0E6FF7AEC04F0E552E5520AD0E8
:104BA000020EDBCFE6FF030EDBCFE6FF42EC34F074
:104BB000E552E5524FD062EC28F04CD0AFEC0EF04D
:104BC00014EC12F047D0550EE66E69EC36F0E55263
:104BD000AA0EE66E7AEC37F0E5523CD085948590CB
:104BE00085928596859A9492000EE66EE66A42EC6E
:104BF00034F0E552E552A4AAFED7D0EC50F0E76EAF
:104C0000010EE7CFDBFF8584858085828586858AD6
:104C10009482640EE66EE66A42EC34F0E552E552A8
:104C200019D0DF6ADF5011E10E01065102E08586DE
:104C300001D08596A4AA08D0D0EC50F0E76E010E02
:104C4000E7CFDBFF010EDF6EEDD704D0010EDF6E84
:104C500001D000D0B2EF20F0F56E040EE15C02E26C
:104C6000E16AE552E16EF550E552E5CFDAFFE7CFB4
:104C7000D9FF1200D9CFE6FFDACFE6FFE1CFD9FFA7
:104C8000E2CFDAFFE652E652E652E652FA0EDBCF08
:104C900000F0FB0EDBCF01F0FC0EDBCF02F0FD0ECF
:104CA000DBCF03F0376A386AC80E396E420E3A6EAF
:104CB00000C032F001C033F002C034F003C035F060
:104CC00021EC3FF0010A07E1DE6ADE6ADE6ADD6A96
:104CD000DD52DD52D0D1FA0EDBCF00F0FB0EDBCF80
:104CE00001F0FC0EDBCF02F0FD0EDBCF03F0376AE4
:104CF000386AC80E396E420E3A6E00C032F001C0FA
:104D000033F002C034F003C035F028EC3FF0010A64
:104D100001E0D9D0376A386A800E396EBF0E3A6E1C
:104D200000C232F001C233F002C234F003C235F0E7
:104D3000B6EC3DF032C004F033C005F034C006F0EC
:104D400035C007F004C0E6FF05C0E6FF06C0E6FF79
:104D500007C0E6FF186A196AC80E1A6E420E1B6E6B
:104D6000FA0EDBCF1CF0FB0EDBCF1DF0FC0EDBCF11
:104D70001EF0FD0EDBCF1FF01CC037F01DC038F059
:104D80001EC039F01FC03AF018C032F019C033F01D
:104D90001AC034F01BC035F0CCEC3CF032C014F03B
:104DA00033C015F034C016F035C017F014C037F01A
:104DB00015C038F016C039F017C03AF008C232F00A
:104DC00009C233F00AC234F00BC235F0B6EC3DF044
:104DD00032C010F033C011F034C012F035C013F0FF
:104DE00010C037F011C038F012C039F013C03AF0DB
:104DF0000CC232F00DC233F00EC234F00FC235F0E7
:104E0000CCEC3CF032C00CF033C00DF034C00EF0EE
:104E100035C00FF00CC0E6FF0DC0E6FF0EC0E6FF88
:104E20000FC0E6FF47EC43F0E552E552E552E5528C
:104E3000E552E7CF07F0E552E7CF06F0E552E7CFBE
:104E400005F0E552E7CF04F031C008F032C009F0B8
:104E500033C00AF034C00BF008C037F009C038F096
:104E60000AC039F00BC03AF004C032F005C033F08C
:104E700006C034F007C035F0CDEC3CF032C000F095
:104E800033C001F034C002F035C003F004C237F083
:104E900005C238F006C239F007C23AF000C032F05D
:104EA00001C033F002C034F003C035F063EC3DF0D4
:104EB00032C0DEFF33C0DEFF34C0DEFF35C0DDFFB1
:104EC000DD52DD52D8D0376A386A800E396EBF0E97
:104ED0003A6E00C232F001C233F002C234F003C2B3
:104EE00035F0B6EC3DF032C004F033C005F034C00C
:104EF00006F035C007F004C0E6FF05C0E6FF06C0B7
:104F0000E6FF07C0E6FF186A196AC80E1A6E420E5D
:104F10001B6EFA0EDBCF1CF0FB0EDBCF1DF0FC0E80
:104F2000DBCF1EF0FD0EDBCF1FF01CC037F01DC025
:104F300038F01EC039F01FC03AF018C032F019C066
:104F400033F01AC034F01BC035F0CCEC3CF032C06A
:104F500014F033C015F034C016F035C017F014C08B
:104F600037F015C038F016C039F017C03AF008C253
:104F700032F009C233F00AC234F00BC235F0B6EC9D
:104F80003DF032C010F033C011F034C012F035C023
:104F900013F010C037F011C038F012C039F013C050
:104FA0003AF00CC232F00DC233F00EC234F00FC230
:104FB00035F0CCEC3CF032C00CF033C00DF034C016
:104FC0000EF035C00FF00CC0E6FF0DC0E6FF0EC0BE
:104FD000E6FF0FC0E6FF47EC43F0E552E552E5522D
:104FE000E552E552E7CF07F0E552E7CF06F0E5528C
:104FF000E7CF05F0E552E7CF04F031C008F032C04A
:1050000009F033C00AF034C00BF008C037F009C013
:1050100038F00AC039F00BC03AF004C032F005C0D5
:1050200033F006C034F007C035F0CDEC3CF032C0B0
:1050300000F033C001F034C002F035C003F004C208
:1050400037F005C238F006C239F007C23AF000C0A6
:1050500032F001C033F002C034F003C035F063EC2D
:105060003DF032C0DEFF33C0DEFF34C0DEFF35C0AE
:10507000DDFFDD52DD52DECF31F0DECF32F0DECFAC
:1050800033F0DDCF34F0DD52DD5200D0F56E040E8A
:10509000E15C02E2E16AE552E16EF550E552E5CFEE
:1050A000DAFFE7CFD9FF1200950E006E600E016E99
:1050B000026A00C0E6FF01C0E6FF7AEC04F0E552A8
:1050C000E5521200D9CFE6FFDACFE6FFE1CFD9FFF4
:1050D000E2CFDAFF060EE12402E3E168E652E16E78
:1050E000580E006E600E016E026A00C0E6FF01C03D
:1050F000E6FF7AEC04F0E552E552A4AAFED7D0EC24
:1051000050F0E76E010EE7CFDBFF3F0E006E600E42
:10511000016E026A00C0E6FF01C0E6FF7AEC04F00F
:10512000E552E552DF6ADFCF00F0080EE76E0018A7
:10513000E8AE02D0E73402D0E750005C0CE22CEC81
:105140001EF0F3CF00F0F4CF01F00050011001E1A8
:10515000F6D7DF2AE8D7280E006E600E016E026ACD
:1051600000C0E6FF01C0E6FF7AEC04F0E552E5522C
:10517000020EDB6A030EDB6A040EDB6A050EDB6AD5
:10518000DF6ADFCF00F0400EE76E0018E8AE02D015
:10519000E73402D0E750005C01E390D02CEC1EF025
:1051A000F3CF00F0F4CF01F00050011001E1F6D789
:1051B000000100016351800B6DE1000100016751A6
:1051C000800B68E1D950020FE96E000EDA20EA6E1A
:1051D000EE5000016825006EEE5000016921016E5D
:1051E000EE5000016A21026EEE5000016B21036E49
:1051F00000C0E6FF01C0E6FF02C0E6FF03C0E6FF15
:1052000068C0E6FF69C0E6FF6AC0E6FF6BC0E6FF64
:10521000D950020FE96E000EDA20EA6EEECFE6FFFB
:10522000EECFE6FFEECFE6FFEFCFE6FF110E046E06
:10523000600E056E066A04C0E6FF05C0E6FF06C004
:10524000E6FF740EE66E000EE66E0FEC4EF0F56EA5
:10525000110EE15C02E2E16AE552E16EF550740E76
:10526000E66E000EE66E53EC04F0E552E552D950BE
:10527000020FE96E000EDA20EA6E00016851EE2698
:1052800000016951EE2200016A51EE2200016B51CA
:10529000EE2212D0030E006E600E016E026A00C094
:1052A000E6FF01C0E6FF7AEC04F0E552E552DFCFFD
:1052B00000F0003401E2DF06DF2A63D7020EDBCF05
:1052C00000F0030EDBCF01F0040EDBCF02F0050E81
:1052D000DBCF03F0060ED8900332023201320032E7
:1052E000E806F9E100C0E6FF01C0E6FF02C0E6FF04
:1052F00003C0E6FFD950020FE96E000EDA20EA6E15
:10530000EECFE6FFEECFE6FFEECFE6FFEFCFE6FF14
:10531000EF0E046E5F0E056E066A04C0E6FF05C060
:10532000E6FF06C0E6FF740EE66E000EE66E0FECBA
:105330004EF0F56E0D0EE15C02E2E16AE552E16EBF
:10534000F550740EE66E000EE66E53EC04F0E55276
:10535000E552D950020FE96E000EDA20EA6E060E11
:10536000E76ED890030EEB32020EEB32010EEB32F9
:10537000EF32E706F6E1046A056AC80E066E4C0EC7
:10538000076E020EDBCF0CF0030EDBCF0DF0040E28
:10539000DBCF0EF0050EDBCF0FF00CC031F00DC0EF
:1053A00032F00EC033F00FC034F0B1EC3CF032C03C
:1053B00008F033C009F034C00AF035C00BF008C063
:1053C00037F009C038F00AC039F00BC03AF004C019
:1053D00032F005C033F006C034F007C035F063EC9E
:1053E0003DF032C000F033C001F034C002F035C0EF
:1053F00003F0376A386AC80E396E420E3A6E00C042
:1054000032F001C033F002C034F003C035F0CCEC10
:105410003CF032C037F233C038F234C039F235C014
:105420003AF2D950020FE96E000EDA20EA6EEECFA2
:10543000E6FFEECFE6FFEECFE6FFEFCFE6FFCE0EC4
:10544000006E5F0E016E026A00C0E6FF01C0E6FF5B
:1054500002C0E6FF740EE66E000EE66E0FEC4EF034
:10546000F56E090EE15C02E2E16AE552E16EF5508B
:10547000740EE66E000EE66E53EC04F0E552E55253
:1054800037C2E6FF38C2E6FF39C2E6FF3AC2E6FF9E
:10549000740EE66E000EE66E74EC3BF0F56E060ED2
:1054A000E15C02E2E16AE552E16EF550B70E006E92
:1054B0005F0E016E026A00C0E6FF01C0E6FF7AECF3
:1054C00004F0E552E552A4AAFED7D0EC50F0E76E06
:1054D000010EE7CFDBFFDF6AA450200B01E08AD08A
:1054E000DFCF00F00A0EE76E0018E8AE02D0E73416
:1054F00002D0E750005C01E37DD02CEC1EF0F3CF2E
:1055000000F0F4CF01F00050011001E1F6D722ECD9
:105510001BF045EC1FF0376A386A340E396E420EC4
:105520003A6E6CC032F06DC033F06EC034F06FC0B4
:1055300035F0CCEC3CF032C004F033C005F034C0A0
:1055400006F035C007F004C0E6FF05C0E6FF06C060
:10555000E6FF07C0E6FF96EC4FF0E552E552E55254
:10556000E55231C000F032C001F033C002F034C067
:1055700003F0CD0E376ECC0E386ECC0E396E3D0E6C
:105580003A6E00C032F001C033F002C034F003C004
:1055900035F031EC3FF0010A1CE1DF2ADFCF00F0EB
:1055A0000A0EE76E0018E8AE02D0E73402D0E750EA
:1055B000005C0EE3980E006E5F0E016E026A00C082
:1055C000E6FF01C0E6FF7AEC04F0E552E55212D0A6
:1055D00001D0DF6AC80EE66E5DEC51F0E552C80EF0
:1055E000E66E5DEC51F0E552C80EE66E5DEC51F0F2
:1055F000E55272D7D0EC50F0E76E010EE7CFDBFF3B
:10560000800E006E5F0E016E026A00C0E6FF01C0F0
:10561000E6FF7AEC04F0E552E552A4AAFED7D0ECFE
:1056200050F0E76E010EE7CFDBFFDF6AA4BA7DD052
:105630002CEC1EF0F3CF00F0F4CF01F0005001107D
:1056400001E1F6D722EC1BF045EC1FF0376A386A0F
:10565000700E396E410E3A6E6CC032F06DC033F090
:105660006EC034F06FC035F0CDEC3CF032C004F0C9
:1056700033C005F034C006F035C007F004C0E6FFC3
:1056800005C0E6FF06C0E6FF07C0E6FF96EC4FF058
:10569000E552E552E552E55231C000F032C001F06A
:1056A00033C002F034C003F0CD0E376ECC0E386E2E
:1056B000CC0E396E3D0E3A6E00C032F001C033F0B0
:1056C00002C034F003C035F031EC3FF0010A1CE1B8
:1056D000DF2ADFCF00F00A0EE76E0018E8AE02D036
:1056E000E73402D0E750005C0EE3980E006E5F0EC8
:1056F000016E026A00C0E6FF01C0E6FF7AEC04F02A
:10570000E552E55212D001D0DF6AC80EE66E5DECBC
:1057100051F0E552C80EE66E5DEC51F0E552C80E50
:10572000E66E5DEC51F0E55281D7D0EC50F0E76EBB
:10573000010EE7CFDBFF94EC48F0F56E060EE15C5E
:1057400002E2E16AE552E16EF550E552E5CFDAFF9B
:10575000E7CFD9FF12000D0A53747275637420539A
:10576000697A653A2025640D0A435243206C656EC0
:105770006774683A2025640D0A4352433A20307812
:1057800025303458000D0A53746F72696E672063B8
:10579000616C6962726174696F6E2076616C7565A7
:1057A00073000D0A43616C6962726174696F6E20E7
:1057B00043524331362050617373656421000D0AF2
:1057C00043616C6962726174696F6E204352433148
:1057D00036204661696C656421000D0A4352433AE4
:1057E00020307825303458000D0A496E6465783AC7
:1057F0002025642C20446174612030782530325893
:10580000000D0A0A4C6F6164696E672063616C6900
:1058100062726174696F6E2076616C756573000DDC
:105820000A5254445F5245463A20000D0A546F6FA5
:105830002068696768000D0A56616C75653A202515
:1058400064000D0A456E746572206120332D646911
:105850006769742064757479206379636C652028A6
:105860003030302D3130302920666F7220746865F9
:10587000205353523A20000D0A42757A7A6572001D
:105880000D0A52656D6F74652052756E20496E70F9
:105890007574000D0A35302F3630487A20496E7005
:1058A0007574000D0A53657420496E707574000D8F
:1058B0000A52756E20696E707574000D0A50756D10
:1058C00070204F7665726C6F616420496E707574DC
:1058D000000D0A4C6576656C20416C61726D204943
:1058E0006E707574000D0A4C6F772050726573737B
:1058F00075726520496E707574000D0A4869676895
:1059000020507265737375726520496E70757400EE
:105910000D0A4C6576656C204661756C7420496E85
:105920007075740020496E6163746976650020416A
:105930006374697665000D0A466C6F7720416C616F
:10594000726D20496E707574000D0A512E205175CC
:105950006974000D0A4A2E2052656D6F74652052DD
:10596000756E20496E707574000D0A492E20353011
:105970002F3630487A20496E707574000D0A482E13
:105980002053657420496E707574000D0A472E20EF
:1059900052756E20496E707574000D0A462E2050A7
:1059A000756D70204F7665726C6F616420496E7002
:1059B0007574000D0A452E204C6576656C20416C8F
:1059C00061726D20496E707574000D0A442E204C72
:1059D0006F7720507265737375726520496E7075AC
:1059E00074000D0A432E2048696768205072657361
:1059F0007375726520496E707574000D0A422E2011
:105A00004C6576656C204661756C7420496E7075C6
:105A100074000D0A0A412E20466C6F7720416C619C
:105A2000726D20496E707574000D0A54656D70209A
:105A3000416C61726D204F6666000D0A54656D7091
:105A400020416C61726D204F6E000D0A4D61696ED0
:105A500020436F6E746163746F72204F6666000D31
:105A60000A4D61696E20436F6E746163746F7220BA
:105A70004F6E000D0A466C6F7720416C61726D208D
:105A80004F6666000D0A466C6F7720416C61726D3F
:105A9000204F6E000D0A4C6576656C204661756C72
:105AA00074204F6666000D0A4C6576656C20466171
:105AB000756C74204F6E000D0A4C6576656C204144
:105AC0006C61726D204F6666000D0A4C6576656CE0
:105AD00020416C61726D204F6E000D0A512E202006
:105AE0002051756974000D0A452F652E2054656D8F
:105AF0007020416C61726D204F6E2F4F6666000DF5
:105B00000A442F642E204D61696E20436F6E7461CC
:105B100063746F72204F6E2F4F6666000D0A432F1D
:105B2000632E20466C6F7720416C61726D204F6E42
:105B30002F4F6666000D0A422F622E204C65766557
:105B40006C204661756C74204F6E2F4F6666000D99
:105B50000A0A412F612E204C6576656C20416C61EC
:105B6000726D204F6E2F4F6666000D0A4A2E20522E
:105B7000656D6F746520496E7075742044422F46C0
:105B8000696C742054657374000D0A492E204375A6
:105B90007272656E742054657374000D0A482E206D
:105BA00054657374204652414D000D0A472E204C17
:105BB0006F61642044656661756C742050494400CF
:105BC0000D0A462E2043616C2052544420496E70C9
:105BD0007574000D0A452E2054657374205353527A
:105BE000204F7574707574000D0A442E205465732F
:105BF000742042757A7A6572000D0A432E20526530
:105C000061642052544420496E707574000D0A423C
:105C10002E2054657374204F70746F20496E707518
:105C20007473000D0A0A412E205465737420526566
:105C30006C6179204F757470757473000D0A446936
:105C400061676E6F73746963205574696C697479E8
:105C5000000D0A52656164696E6720626C6F636B48
:105C6000202564206F66202564000D0A5772697430
:105C7000696E6720626C6F636B202564206F6620FD
:105C80002564000D0A2564206572726F72732066A8
:105C90006F756E64002530325820000D0A000D0A21
:105CA000095374617475733A2025303258000D0A17
:105CB000494E49543A204652414D000D0A64776FCF
:105CC00072643A202530386C582C0D0A627974655C
:105CD0005B305D3A20253032582C0D0A62797465AC
:105CE0005B315D3A20253032582C0D0A627974659B
:105CF0005B325D3A20253032582C0D0A627974658A
:105D00005B335D3A20253032580D0A656F633A20C7
:105D1000253032580D0A63683A20253032580D0A72
:105D20007369673A20253032580D0A6578723A2037
:105D3000253032580D0A64617461683A202530328A
:105D4000580D0A646174616D3A20253032580D0A8D
:105D5000646174616C3A20253032580D0A706164B8
:105D60003A20253032580D0A000D0A525444205270
:105D700061773A2030782530386C58095363616C6C
:105D800065643A20000D0A0A4C5443323432322002
:105D9000696E6974002530336C6400256C642E00D4
:105DA0000D0A0A53504920696E6974285350495F9F
:105DB000464F53435F31362C204D4F44455F3030C2
:105DC0002C20534D504D494429000D0A2A2A2A2AD5
:105DD0002A2A2A2A2A2A2A2A2A2A2A2A2A2A2A2A23
:105DE0002A2A2A2A2A2A2A2A2A2A2A2A2A2A2A2A13
:105DF0002A2A000D0A52656C656173652054696D2D
:105E0000653A20253032583A253032583A2530321A
:105E100058000D0A52656C656173652044617465B4
:105E20003A20253032582F253032582F253032581D
:105E3000000D0A46572076657273696F6E3A202509
:105E40003032582E253032582E25303458000D0A65
:105E50004368696C6C6572000D0A4C7964616C6C06
:105E6000000D0A0A2A2A2A2A2A2A2A2A2A2A2A2A19
:105E70002A2A2A2A2A2A2A2A2A2A2A2A2A2A2A2A82
:105E80002A2A2A2A2A2A2A2A2A2A00097274645FBC
:105E90007265663D00096F75747075743D0009691F
:105EA0006E7075743D000D0A7461726765743D0013
:105EB0000D0A53746F72696E672050494420676100
:105EC000696E73000D0A5049442043524331362015
:105ED00050617373656421000D0A4C6F6164696ED3
:105EE0006720504944206761696E732066726F6D48
:105EF00020706167652032000D0A504944204352EA
:105F0000433136204661696C656421000D0A4352B5
:105F1000433A20307825303458000D0A496E6465C4
:105F2000783A2025642C2044617461203078253033
:105F30003258000D0A0A4C6F6164696E672050493F
:105F400044206761696E732066726F6D20706167AF
:105F500065203100096172773D2000096B643D20A6
:105F600000096B693D20000D0A5049443A206B70CE
:105F70003D20000D0A0A50494420696E69742000D2
:105F80000D0A5365742073696D756C61746F7220AE
:105F9000746F202D313543000D0A52544420636143
:105FA0006C69627261746564207375636365737391
:105FB00066756C6C7921000D0A5365742073696DE8
:105FC000756C61746F7220746F20343543000D0A54
:105FD000283130343835373630302E30202F2025D8
:105FE0006C6429202D203130302E30203D20000DD2
:105FF0000A53756D3A20256C64204176673A202556
:106000006C64000D0A4261642073616D706C6521DF
:10601000000D0A53756D3A20256C64202B20256CE9
:1060200064203D20256C64000D0A4176657261672D
:10603000696E672036342073616D706C6573000D76
:106040000A5468726F77696E67206F757420382004
:1060500073616D706C6573000D0A436F6E6E6563DE
:106060007420746865205254442073696D756C61A6
:10607000746F7220746F2052544420696E7075746E
:1060800020616E642073657420697420746F2074BD
:106090006F203043000D0A0A52544420696E69741F
:1060A00000000E01006B0E01016B0E01026B0E0170
:1060B000036B0E01046BE66A140EE66E050EE66EC7
:1060C0000E0EE66EFCD9E552E552E552E552E66A5F
:1060D000140EE66E0B0EE66E0E0EE66EF0D9E5526D
:1060E000E552E552E552010EE66E280EE66E110EFF
:1060F000E66E0E0EE66EE3D9E552E552E552E55244
:10610000010EE66E280EE66E170EE66E0E0EE66EB9
:10611000D6D9E552E552E552E552010EE66E280E5B
:10612000E66E1D0EE66E0E0EE66EC9D9E552E5521C
:10613000E552E552010EE66E050EE66E230EE66EA2
:106140000E0EE66EBCD9E552E552E552E552010E5F
:10615000E66E050EE66E290EE66E0E0EE66EAFD901
:10616000E552E552E552E552E66A280EE66E2F0E3C
:10617000E66E0E0EE66EA3D9E552E552E552E55203
:10618000E66A140EE66E3B0EE66E0E0EE66E97D9CC
:10619000E552E552E552E552E66A140EE66E350E1A
:1061A000E66E0E0EE66E8BD9E552E552E552E552EB
:1061B000010EE66E140EE66E410EE66E0E0EE66EF3
:1061C0007ED9E552E552E552E552010EE66E140E17
:1061D000E66E470EE66E0E0EE66E71D9E552E5529A
:1061E000E552E552010EE66E140EE66E4D0EE66EB9
:1061F0000E0EE66E64D9E552E552E552E552010E07
:10620000E66E140EE66E530EE66E0E0EE66E57D96F
:10621000E552E552E552E5520F0EE66E590EE66E76
:106220000E0EE66E99D9E552E552E5520F0EE66E76
:106230005D0EE66E0E0EE66E8FD9E552E552E55222
:106240000F0EE66E610EE66E0E0EE66E85D9E55215
:10625000E552E5520F0EE66E650EE66E0E0EE66E28
:106260007BD9E552E552E5520F0EE66E690EE66EF9
:106270000E0EE66E71D9E552E552E5520F0EE66E4E
:106280006D0EE66E0E0EE66E67D9E552E552E552EA
:106290000F0EE66E710EE66E0E0EE66E5DD9E552DD
:1062A000E552E5520F0EE66E750EE66E0E0EE66EC8
:1062B00053D9E552E552E5520F0EE66E7D0EE66EBD
:1062C0000E0EE66E49D9E552E552E5520F0EE66E26
:1062D000790EE66E0E0EE66E3FD9E552E552E552B6
:1062E00012008650080B01E0010E0E01596F865016
:1062F000010B0E015D6F8350800B01E0010E0E015A
:10630000616F8350400B01E0010E0E01656F8350F9
:10631000040B01E0010E0E01696F8350200B01E0B8
:10632000010E0E016D6F8350100B01E0010E0E0186
:10633000716F8350080B01E0010E0E01756F8350E1
:10634000010B0E017D6F8350020B01E0010E0E0167
:10635000796F590EE66E0E0EE66E33D9E552E552B0
:106360005D0EE66E0E0EE66E2CD9E552E552610E1C
:10637000E66E0E0EE66E25D9E552E552650EE66E26
:106380000E0EE66E1ED9E552E552690EE66E0E0E51
:10639000E66E17D9E552E5526D0EE66E0E0EE66E0C
:1063A00010D9E552E552710EE66E0E0EE66E09D971
:1063B000E552E552750EE66E0E0EE66E02D9E55216
:1063C000E5527D0EE66E0E0EE66EFBD8E552E55206
:1063D000790EE66E0E0EE66EF4D8E552E552010136
:1063E000FE2B320E0101FE5D69E35ACE05FE5ECE44
:1063F0000BFE62CE11FE66CE17FE6ACE1DFE6ECE7D
:1064000023FE72CE29FE76CE2FFE7ECE3BFE7ACEC6
:1064100035FE050EE66E0E0EE66E50D9E552E552DB
:1064200000090BE00E01065105E0C80E0001F46FF3
:10643000F56B03D00001F46BF56B0B0EE66E0E0EE0
:10644000E66E3CD9E552E552110EE66E0E0EE66E92
:1064500035D9E552E552170EE66E0E0EE66E2ED9D0
:10646000E552E5521D0EE66E0E0EE66E27D9E55298
:10647000E552230EE66E0E0EE66E20D9E552E55289
:10648000290EE66E0E0EE66E19D9E552E5522F0E74
:10649000E66E0E0EE66E12D9E552E5523B0EE66E42
:1064A0000E0EE66E0BD9E552E552350EE66E0E0E77
:1064B000E66E04D9E552E5520101FE6B1200D9CF18
:1064C000E6FFDACFE6FFE1CFD9FFE2CFDAFFFC0E3D
:1064D000DBCFE9FFFD0EDBCFEAFFEF6AFC0EDBCF7F
:1064E000E9FFFD0EDBCFEAFFEE52EF6AFC0EDBCFD9
:1064F000E9FFFD0EDBCFEAFF020EE926000EEA22DD
:10650000FA0EDBCFEFFFFC0EDBCFE9FFFD0EDBCF9A
:10651000EAFF040EE926000EEA22EF6AFC0EDBCF4A
:10652000E9FFFD0EDBCFEAFF030EE926000EEA22AB
:10653000EF6AFC0EDBCFE9FFFD0EDBCFEAFF050EB5
:10654000E926000EEA22FB0EDBCFEFFFE552E5CF96
:10655000DAFFE7CFD9FF1200D9CFE6FFDACFE6FFA7
:10656000E1CFD9FFE2CFDAFFFC0EDBCFE9FFFD0E72
:10657000DBCFEAFFEF6AFC0EDBCFE9FFFD0EDBCFDE
:10658000EAFFEE52EF6AFC0EDBCFE9FFFD0EDBCF38
:10659000EAFF030EE926000EEA22FB0EDBCFEFFF37
:1065A000FC0EDBCFE9FFFD0EDBCFEAFF020EE92692
:1065B000000EEA22EF6AE552E5CFDAFFE7CFD9FF16
:1065C0001200D9CFE6FFDACFE6FFE1CFD9FFE2CF65
:1065D000DAFFFC0EDBCFE9FFFD0EDBCFEAFF020E98
:1065E000E926000EEA22EF9EEF46FC0EDBCFE9FF24
:1065F000FD0EDBCFEAFFEFCF00F0FC0EDBCFE9FFB3
:10660000FD0EDBCFEAFF020EE926000EEA22005063
:10661000EF12FC0EDBCFE9FFFD0EDBCFEAFF030E2E
:10662000E926000EEA22EFCF00F0FC0EDBCFE9FFF7
:10663000FD0EDBCFEAFF020EE926000EEA22005033
:10664000EF16FC0EDBCFE9FFFD0EDBCFEAFF020EFB
:10665000E926000EEA22EFCF00F0FC0EDBCFE9FFC7
:10666000FD0EDBCFEAFF030EE926000EEA22EF5013
:10667000005C0AE1FC0EDBCFE9FFFD0EDBCFEAFF99
:10668000EE52010EEF6E14D0FC0EDBCFE9FFFD0ED3
:10669000DBCFEAFF020EE926000EEA22EF5008E106
:1066A000FC0EDBCFE9FFFD0EDBCFEAFFEE52EF6A17
:1066B000E552E5CFDAFFE7CFD9FF1200D9CFE6FFE9
:1066C000DACFE6FFE1CFD9FFE2CFDAFFE652DF6AA9
:1066D000FC0EDBCFE9FFFD0EDBCFEAFFEE52EF5001
:1066E0005CE0FC0EDBCFE9FFFD0EDBCFEAFF030E23
:1066F000E926000EEA22EF6AFC0EDBCFE9FFFD0E71
:10670000DBCFEAFFEFCF00F0FC0EDBCFE9FFFD0EA1
:10671000DBCFEAFF020EE926000EEA22EF50005C12
:1067200030E0FC0EDBCFE9FFFD0EDBCFEAFF040E0D
:10673000E926000EEA22EFCF00F0FC0EDBCFE9FFE6
:10674000FD0EDBCFEAFF050EE926000EEA22EF5030
:10675000005C0CE2FC0EDBCFE9FFFD0EDBCFEAFFB5
:10676000040EE926000EEA22EF2A0AD0FC0EDBCF47
:10677000E9FFFD0EDBCFEAFFEE52EF6A010EDF6E9E
:106780000BD0FC0EDBCFE9FFFD0EDBCFEAFF040EE2
:10679000E926000EEA22EF6A5CD0FC0EDBCFE9FFAF
:1067A000FD0EDBCFEAFF040EE926000EEA22EF6AB7
:1067B000FC0EDBCFE9FFFD0EDBCFEAFFEFCF00F0F1
:1067C000FC0EDBCFE9FFFD0EDBCFEAFF020EE92670
:1067D000000EEA22EF50005C31E1FC0EDBCFE9FF56
:1067E000FD0EDBCFEAFF030EE926000EEA22EFCF13
:1067F00000F0FC0EDBCFE9FFFD0EDBCFEAFF050E5C
:10680000E926000EEA22EF50005C0CE2FC0EDBCF22
:10681000E9FFFD0EDBCFEAFF030EE926000EEA22B8
:10682000EF2A0BD0FC0EDBCFE9FFFD0EDBCFEAFF3A
:10683000EE52010EEF6E010EDF6E0BD0FC0EDBCFC1
:10684000E9FFFD0EDBCFEAFF030EE926000EEA2288
:10685000EF6ADF5000D0E552E552E5CFDAFFE7CF2F
:10686000D9FF12000E01816B826B0E01836B846B6A
:106870000E01856B866B000EE66EE66A03D8E55264
:10688000E5521200D9CFE6FFDACFE6FFE1CFD9FF1C
:10689000E2CFDAFF050E336E346AFC0EDBCF38F040
:1068A000FD0EDBCF39F076EC3EF031C085FE32C014
:1068B00086FE0E01040E855D000E865903E20E0170
:1068C000856B866BE552E5CFDAFFE7CFD9FF120083
:1068D0000E0183510E01815D0E0184510E0182591A
:1068E00002E2858C01D0859C0E0181CE00F082CE23
:1068F00001F0812B000E8223F40E005C010E015882
:1069000007E30E01816B826B85CE83FE86CE84FE0B
:1069100012000E01005102E0859201D085820E0125
:10692000015102E0859001D085800E01025102E004
:10693000859401D085840E01035102E0859A01D02F
:10694000858A0E01045102E0859601D085861200E9
:10695000D9CFE6FFDACFE6FFE1CFD9FFE2CFDAFF0A
:10696000E652AE0E006E5C0E016E026A00C0E6FFDB
:1069700001C0E6FF7AEC04F0E552E5528484040E8F
:10698000E66EDDEC51F0E5528494050EE66E45ECC2
:1069900051F0E55210EC52F0DF6E8484DFCFE6FF59
:1069A000E66A9E0E006E5C0E016E026A00C0E6FF93
:1069B00001C0E6FF02C0E6FF740EE66E000EE66E52
:1069C0000FEC4EF0F56E070EE15C02E2E16AE55273
:1069D000E16EF550740EE66E000EE66E53EC04F0B8
:1069E000E552E552010EF36EF46A00D0E552E5522D
:1069F000E5CFDAFFE7CFD9FF1200D9CFE6FFDACF34
:106A0000E6FFE1CFD9FFE2CFDAFFE6528488849433
:106A1000060EE66E45EC51F0E55284848494020E35
:106A2000E66E45EC51F0E552FC0EDBCF00F0FD0EBA
:106A3000DBCF01F001C000F0016A0050E66E45ECCA
:106A400051F0E552FC0EDBCFE6FF45EC51F0E5528C
:106A5000FB0EDBCFE6FF45EC51F0E55284848494D5
:106A6000050EE66E45EC51F0E55210EC52F0DF6E8B
:106A70008484DFA001D0F3D78494040EE66E45EC45
:106A800051F0E55284848498010EF36EF46A00D0CC
:106A9000E552E552E5CFDAFFE7CFD9FF1200D9CFB3
:106AA000E6FFDACFE6FFE1CFD9FFE2CFDAFFE65229
:106AB000E652DF6AF80EDBCF00F0F90EDBCF01F013
:106AC000013404E200502008000E015403E2F36A8E
:106AD000F46A5BD084888494060EE66E45EC51F02F
:106AE000E55284848494020EE66E45EC51F0E55242
:106AF000FC0EDBCF00F0FD0EDBCF01F001C000F09B
:106B0000016A0050E66E45EC51F0E552FC0EDBCF19
:106B1000E6FF45EC51F0E552F80EDBCF00F0DB0666
:106B2000F90EDBCF01F001E2DB06005001100FE0AF
:106B3000FA0EDBCFE9FFDB2AFB0EDBCFEAFF01E336
:106B4000DB2AEF50E66E45EC51F0E552E5D7848440
:106B5000020EE66EDDEC51F0E5528494040EE66E12
:106B600045EC51F0E55284848498DFCF00F00F0E9D
:106B7000E76E0018E8AE02D0E73402D0E750005CC0
:106B800000E3010EF36EF46A00D0E552E552E552DF
:106B9000E5CFDAFFE7CFD9FF1200D9CFE6FFDACF92
:106BA000E6FFE1CFD9FFE2CFDAFFE6528494030E8D
:106BB000E66E45EC51F0E552FC0EDBCF00F0FD0E29
:106BC000DBCF01F001C000F0016A0050E66E45EC39
:106BD00051F0E552FF0EE76EFC0EDBCF00F0FD0E2C
:106BE000DBCF01F0E7500016016A0050E66E45EC7D
:106BF00051F0E55210EC52F0DF6E8484DF5000D08B
:106C0000E552E552E5CFDAFFE7CFD9FF1200D9CF41
:106C1000E6FFDACFE6FFE1CFD9FFE2CFDAFFE652B7
:106C2000E652E6528494030EE66E45EC51F0E552CE
:106C3000FC0EDBCF00F0FD0EDBCF01F001C000F059
:106C4000016A0050E66E45EC51F0E552FF0EE76E2A
:106C5000FC0EDBCF00F0FD0EDBCF01F0E75000169D
:106C6000016A0050E66E45EC51F0E552DE6ADD6ADD
:106C7000DECF00F0DDCF01F0F80EDBCF02F0F90E31
:106C8000DBCF03F00250005C0350015814E210EC1B
:106C900052F0E66EFA0EDBCFE9FFDB2AFB0EDBCF0C
:106CA000EAFF01E3DB2AE552E750EF6EDF2A010E2F
:106CB00001E3DB2ADDD78484010EF36EF46A00D091
:106CC000E552E552E552E552E5CFDAFFE7CFD9FFCD
:106CD0001200D9CFE6FFDACFE6FFE1CFD9FFE2CF4E
:106CE000DAFF070EE12402E3E168E652E16E010EED
:106CF000DB6A020EDB6A030EDB6A040EDB6A030E3C
:106D0000DBCF00F0040EDBCF01F0D890015004E699
:106D1000200E005C000E015840E2050EDB6A060EF4
:106D2000DB6A050EDBCF00F0060EDBCF01F0D8905A
:106D3000015004E6080E005C000E015828E2FD0E2A
:106D4000DBCFE6FF050EDBCF02F0060EDBCF03F054
:106D5000080E336E346A030EDBCF38F0040EDBCF3F
:106D600039F049EC3EF031500224006E32500320DD
:106D7000016E00C0E6FF01C0E6FF3FDEE552E552CE
:106D8000E552050EDB2A060E01E3DB2ACAD7030E05
:106D9000DB2A040E01E3DB2AB2D7030EDB6A040E02
:106DA000DB6A030EDBCF00F0040EDBCF01F0D890DE
:106DB000015004E6000E005C010E015866E2030E6D
:106DC000DBCFE6FF040EDBCFE6FFE7DEE552E55260
:106DD000DF6EFD0EDB50DF5C05E0010EDB2A020EEC
:106DE00001E3DB2A030EDBCF00F0040EDBCF01F062
:106DF000100E386E396A00C033F001C034F023EC55
:106E00003EF02FC000F030C001F0005001100DE145
:106E10009B0E006E5C0E016E026A00C0E6FF01C0B0
:106E2000E6FF7AEC04F0E552E552DFCF00F0016AAC
:106E300000BE016800C0E6FF01C0E6FF950E026ECD
:106E40005C0E036E046A02C0E6FF03C0E6FF04C0E6
:106E5000E6FF740EE66E000EE66E0FEC4EF0F56E79
:106E6000070EE15C02E2E16AE552E16EF550740E54
:106E7000E66E000EE66E53EC04F0E552E552030EAA
:106E8000DB2A040E01E3DB2A8CD7010EDBCFE6FF01
:106E9000020EDBCFE6FF830E006E5C0E016E026A0F
:106EA00000C0E6FF01C0E6FF02C0E6FF740EE66E1A
:106EB000000EE66E0FEC4EF0F56E070EE15C02E29E
:106EC000E16AE552E16EF550740EE66E000EE66E74
:106ED00053EC04F0E552E552F56E070EE15C02E278
:106EE000E16AE552E16EF550E552E5CFDAFFE7CF12
:106EF000D9FF1200D9CFE6FFDACFE6FFE1CFD9FF05
:106F0000E2CFDAFF270EE12402E3E168E652E16E08
:106F1000250EDB6A260EDB6A210EDB6A220EDB6A97
:106F2000210EDBCF00F0220EDBCF01F0200E005C43
:106F3000000E015815E2D9CF00F0DACF01F0210E92
:106F4000DB500024E96E220EDB500120EA6EFD0EBC
:106F5000DBCFEFFF210EDB2A220E01E3DB2AE0D795
:106F6000210EDB6A220EDB6A210EDBCF00F0220E3F
:106F7000DBCF01F0026A036AD8900350000A08E6EA
:106F8000000E005C010E0158000E0258000E03585E
:106F900050E2FF0EE66EE66A210EDBCFE6FF220E20
:106FA000DBCFE6FF6A0E006E5C0E016E026A00C067
:106FB000E6FF01C0E6FF02C0E6FF740EE66E000EBB
:106FC000E66E0FEC4EF0F56E090EE15C02E2E16A4E
:106FD000E552E16EF550740EE66E000EE66E53EC6F
:106FE00004F0E552E552200EE66EE66AD9CFE6FFE0
:106FF000DACFE6FF210EDBCF00F0220EDBCF01F06F
:10700000050ED89000360136E806FBE100C0E6FF29
:1070100001C0E6FF44DDF56E060EE15C02E2E16AC6
:10702000E552E16EF550210EDB2A220E01E3DB2A48
:107030009BD79B0E006E5C0E016E026A00C0E6FFDD
:1070400001C0E6FF7AEC04F0E552E552210EDB6A5E
:10705000220EDB6A210EDBCF00F0220EDBCF01F027
:10706000026A036AD8900350000A08E6000E005C2A
:10707000010E0158000E0258000E035870E2FF0E78
:10708000E66EE66A210EDBCFE6FF220EDBCFE6FFDF
:10709000510E006E5C0E016E026A00C0E6FF01C078
:1070A000E6FF02C0E6FF740EE66E000EE66E0FEC21
:1070B0004EF0F56E090EE15C02E2E16AE552E16E26
:1070C000F550740EE66E000EE66E53EC04F0E552D9
:1070D000E552230EDB6A240EDB6A230EDBCF00F0C1
:1070E000240EDBCF01F0200E005C000E015831E2CF
:1070F000210EDBCF02F0220EDBCF03F0050ED8907D
:1071000002360336E806FBE1230EDB500224006E54
:10711000240EDB500320016E00C0E6FF01C0E6FF35
:107120003CDDE552E552E76E200EE7CFDBFFFD0EBA
:10713000DB50F36E200EDB50F35C05E0250EDB2AFE
:10714000260E01E3DB2A230EDB2A240E01E3DB2AD1
:10715000C4D7210EDB2A220E01E3DB2A7BD7250EC2
:10716000DBCFE6FF260EDBCFE6FF830E006E5C0E64
:10717000016E026A00C0E6FF01C0E6FF02C0E6FF42
:10718000740EE66E000EE66E0FEC4EF0F56E070E16
:10719000E15C02E2E16AE552E16EF550740EE66EE2
:1071A000000EE66E53EC04F0E552E552F56E270E44
:1071B000E15C02E2E16AE552E16EF550E552E5CFAD
:1071C000DAFFE7CFD9FF1200000EE66EE66A0EEC9A
:1071D00051F0E552E552450EE66EAFEC50F0E55247
:1071E000000EE66EE66A0EEC51F0E552E5529D8027
:1071F000D08EF29CF28E12000F0EC16E806A926ADF
:1072000081689368410E826E900E946E83689568D3
:10721000B06A8468966A3F0E856E3F0E8E6E070ECA
:10722000B46E800E976E020E866E0D0E986E120072
:10723000D9CFE6FFDACFE6FFE1CFD9FFE2CFDAFF21
:10724000070EE12402E3E168E652E16E0001F66B0D
:10725000F76B0001F96B0001F86B0001FA6B00019C
:10726000FB6B4EEC49F0C8DF6BEC05F03DEC04F035
:10727000B8EC51F051EC30F032EC34F0610E006EAD
:107280005E0E016E026A00C0E6FF01C0E6FF7AEC06
:1072900004F0E552E552580E006E5E0E016E026A71
:1072A00000C0E6FF01C0E6FF7AEC04F0E552E552CB
:1072B0004E0E006E5E0E016E026A00C0E6FF01C057
:1072C000E6FF7AEC04F0E552E552F20EF66EF7684E
:1072D000010EF86E0900F5CFE6FF0800F5CFE6FFD6
:1072E000F10EF66EF768010EF86E0800F5CF00F0AB
:1072F000016A00BE016800C0E6FF01C0E6FFF00EB3
:10730000F66EF768010EF86E0800F5CF02F0036A1A
:1073100002BE036802C0E6FF03C0E6FF310E046E42
:107320005E0E056E066A04C0E6FF05C0E6FF06C0F5
:10733000E6FF740EE66E000EE66E0FEC4EF0F56E94
:107340000B0EE15C02E2E16AE552E16EF550740E6B
:10735000E66E000EE66E53EC04F0E552E552F60ED2
:10736000F66EF768010EF86E0900F5CFE6FF08002B
:10737000F5CFE6FFF40EF66EF768010EF86E080022
:10738000F5CF00F0016A00BE016800C0E6FF01C051
:10739000E6FFF50EF66EF768010EF86E0800F5CF01
:1073A00002F0036A02BE036802C0E6FF03C0E6FF04
:1073B000120E046E5E0E056E066A04C0E6FF05C07E
:1073C000E6FF06C0E6FF740EE66E000EE66E0FECFA
:1073D0004EF0F56E0B0EE15C02E2E16AE552E16E01
:1073E000F550740EE66E000EE66E53EC04F0E552B6
:1073F000E552FB0EF66EF768010EF86E0800F5CF49
:1074000000F0016A00BE016800C0E6FF01C0E6FFAF
:10741000FA0EF66EF768010EF86E0800F5CF02F06E
:10742000036A02BE036802C0E6FF03C0E6FFF80E6F
:10743000F66EF768010EF86E0800F5CF04F0056AE5
:1074400004BE056804C0E6FF05C0E6FFF30E066E45
:107450005D0E076E086A06C0E6FF07C0E6FF08C0BB
:10746000E6FF740EE66E000EE66E0FEC4EF0F56E63
:107470000B0EE15C02E2E16AE552E16EF550740E3A
:10748000E66E000EE66E53EC04F0E552E552CA0ECD
:10749000006E5D0E016E026A00C0E6FF01C0E6FFED
:1074A0007AEC04F0E552E552A00E006E5D0E016E1E
:1074B000026A00C0E6FF01C0E6FF7AEC04F0E55284
:1074C000E552E66AE66A010EE66E63EC4FF0E552BD
:1074D000E552E552A8EC34F0F3CF00F0F4CF01F020
:1074E000010E001801E1015000E169EC47F05EEC8B
:1074F0000EF0E9EC1AF06AEC45F066DE15EC40F0AF
:107500000001FA5104E00001FA6B25EC40F00101A2
:10751000F25102E1A3EC05F0F3D7F56E070EE15C42
:1075200002E2E16AE552E16EF550E552E5CFDAFF9D
:10753000E7CFD9FF1200E9CFE4FFEACFE4FFF6CFAF
:10754000E4FFF7CFE4FFF5CFE4FFF3CFE4FFF4CFA0
:10755000E4FFFACFE4FF00EE2DF0140EE80403E39D
:10756000EECFE4FFFBD700EE00F0200EE80403E3CB
:10757000EECFE4FFFBD7E6529EA05ED09E90E80ED1
:10758000CF6ECE6A0101F2050CE1ACA206D0849068
:10759000000084920101F26B03D00101020EF26F30
:1075A00008D00101F25105E08490000084920101AD
:1075B000F26B0101F15102E00101F1070101EF510C
:1075C00002E00101EF070001F92B320E0001F95D25
:1075D00018E30001010EFA6F0001F96B0001FC2BAA
:1075E000050E0001FC5D05E30001010EFD6F0001C9
:1075F000FC6B0001F451F51104E00001F407000EEA
:10760000F55B0001F62B000EF7230001E80EF65D96
:10761000030EF75904E30001F66BF76B847671EC07
:1076200031F00001FB51FB2B416E0A0E415C04E37B
:1076300068EC34F00001FB6B9EAA11D0010180516F
:107640003F0802E20101806B01018051802BEA6A50
:10765000400FE96E010EEA22AECFEFFF9E9A9E50D8
:10766000100B1EE09D50100B1BE00101C3510101E6
:10767000C25D12E00101C3513F0802E20101C36B88
:107680000101C351C32BEA6A820FE96E010EEA229F
:10769000EF50AD6E9E9804D00101010EF26F9D98DF
:1076A000A1B0A190E55200EE1FF0200EE80403E324
:1076B000E5CFEDFFFBD700EE40F0140EE80403E346
:1076C000E5CFEDFFFBD7E5CFFAFFE5CFF4FFE5CF40
:1076D000F3FFE5CFF5FFE5CFF7FFE5CFF6FFE5CF09
:1076E000EAFFE5CFE9FF1100D9CFE6FFDACFE6FFE9
:1076F000E1CFD9FFE2CFDAFF080EE12402E3E1682F
:10770000E652E16EF80EDBCF32F0F90EDBCF33F04C
:10771000FA0EDBCF34F0FB0EDBCF35F0EAEC3EF0B7
:1077200031C0DEFF32C0DEFF33C0DEFF34C0DDFF1C
:10773000DD52DD52D9CFE9FFDACFEAFFEECF08F014
:10774000EECF09F0EECF0AF0EFCF0BF0E80E366E79
:10775000030E376E386A396A08C031F009C032F05A
:107760000AC033F00BC034F0F8EC4EF02DC008F036
:107770002EC009F02FC00AF030C00BF0F80EDBCF9E
:1077800004F0F90EDBCF05F0FA0EDBCF06F0FB0EAE
:10779000DBCF07F0376A386A7A0E396E440E3A6EDC
:1077A00004C032F005C033F006C034F007C035F035
:1077B000B6EC3DF0EAEC3EF000010850315C006EA2
:1077C000000109503258016E00010A503358026E10
:1077D00000010B503458036E040E00C0DBFF050E91
:1077E00001C0DBFF060E02C0DBFF070E03C0DBFF9C
:1077F000D950040FE96E000EDA20EA6ED890030E1D
:10780000EB50000A08E6000EEE5C000EEE58000E8B
:10781000EE58000EEE581EE2040EDBCF31F0050EDE
:10782000DBCF32F0060EDBCF33F0070EDBCF34F0C8
:107830003668376838683968F8EC4EF0040E2DC0A9
:10784000DBFF050E2EC0DBFF060E2FC0DBFF070E91
:1078500030C0DBFFD9CFE9FFDACFEAFFEECFE6FF9A
:10786000EECFE6FFEECFE6FFEFCFE6FF9B0E006E1A
:107870005D0E016E026A00C0E6FF01C0E6FF02C0B5
:10788000E6FFFC0EDBCFE6FFFD0EDBCFE6FF0FECE5
:107890004EF0F56E090EE15C02E2E16AE552E16E3E
:1078A000F550FC0EDBCFE6FFFD0EDBCFE6FF53EC21
:1078B00004F0E552E552D950040FE96E000EDA20CB
:1078C000EA6EEECFE6FFEECFE6FFEECFE6FFEFCFBC
:1078D000E6FF950E006E5D0E016E026A00C0E6FFC7
:1078E00001C0E6FF02C0E6FFFC0EDBCFE6FFFD0EA7
:1078F000DBCFE6FF0FEC4EF0F56E090EE15C02E225
:10790000E16AE552E16EF550FC0EDBCFE6FFFD0EBD
:10791000DBCFE6FF53EC04F0E552E552F56E080EBE
:10792000E15C02E2E16AE552E16EF550E552E5CF35
:10793000DAFFE7CFD9FF12003C9E08D03C9E34AE60
:1079400005D0336C341EE86A34223C8E34C02EF0ED
:1079500033C02DF0406A3F6A8E0E2F6E306AABEF57
:107960003FF03C9E0CD03C9E34AE09D0316C321EB0
:10797000331E341EE86A3222332234223C8E34C055
:107980002EF033C02DF032C040F031C03FF09E0EDB
:107990002F6E306AABEF3FF03A7E3C6AE7EC3FF087
:1079A000FFEC3FF03CB68FEF3FF03CA20AD03CAA80
:1079B00003D03CBE8FEF3FF03CA49BEF3FF098EF2D
:1079C0003FF03CAA05D03CAC9BEF3FF098EF3FF076
:1079D0003CA00AD03CA808D03CBE04D03CA402D0B5
:1079E000A4EF3FF0A8EF3FF03F6A306A3A50355CB1
:1079F0003E6E10E332C040F033C02DF034C02EF0A4
:107A000035C03DF037C032F038C033F039C034F003
:107A10003C3A09D037C040F038C02DF039C02EF0C4
:107A20003AC03DF03E6C3C9E3CBC3C8E3DC02FF0CD
:107A30003CB0D7EF3FF01A0E3E60D7EF3FF02F6A11
:107A4000356A3CA408D0326C331E341E351EE86AF9
:107A50003322342235223CAC08D0406C2D1E2E1E21
:107A60002F1EE86A2D222E222F22316A3E5207E075
:107A7000353434323332323231323E2EF9D732504D
:107A8000402633502D2234502E2235502F2231C023
:107A90003FF03C9E2FAE0BD03F6C401E2D1E2E1E85
:107AA0002F1EE86A40222D222E222F223C8E2FA04C
:107AB00006D0D8802E322D3240323F323D2A3DC092
:107AC0002FF0ABEF3FF03C6AE7EC3FF0FFEC3FF00C
:107AD0003CB68FEF3FF03CA205D03CBA8FEF3FF0B1
:107AE00096EF3FF03CBAA2EF3FF03CA005D03CB887
:107AF0008FEF3FF0A2EF3FF03CB896EF3FF0306AD7
:107B00007F0E35242F6EE86A30223A502F5EE86AE5
:107B1000305A1A0E3D6E356A3F6A406A2D6A2E6AE7
:107B20003750325E3850335A3950345A000E355A75
:107B300009E7375032263850332239503422000EAC
:107B4000352201D03F8AD890323633363436353636
:107B5000D8903F3640362D362E363D2EE1D7345064
:107B600033103210D8A43F8AABEF3FF03C6AE7EC09
:107B70003FF0FFEC3FF03CB68FEF3FF03CA205D06A
:107B80003CB88FEF3FF096EF3FF03CAA05D03CB0F9
:107B90008FEF3FF096EF3FF03CB002D03CA802D010
:107BA000A2EF3FF0306A3A5035242F6EE86A302257
:107BB0007E0E2F5EE86A305A3F6A406A2D6A2E6A4E
:107BC00039503402F4CF2EF0F3CF2DF03850340278
:107BD000F3504026F4502D22000E2E22395033024D
:107BE000F3504026F4502D22000E2E22375034023E
:107BF000F3503F26F4504022000E2D222E22385002
:107C00003302F3503F26F4504022000E2D222E2244
:107C100039503202F3503F26F4504022000E2D22FC
:107C20002E2237503302F4503F26000E40222D22E0
:107C30002E2238503202F4503F26000E40222D22D0
:107C40002E22ABEF3FF03B6A39AE2CEF3EF0386CA2
:107C5000391EE86A39223B1E34AE34EF3EF0336CF5
:107C6000341EE86A34223B1EA2EC51F034BE44EFCD
:107C70003EF03BAE000C336C341EE86A34222F6CAD
:107C8000301EE86A3022000C3BBE3BEF3EF03C88E1
:107C9000FF0C34C040F033C03FF033503802F4CF13
:107CA00032F0F3CF31F034503902F4CF34F0F3CF67
:107CB00033F03802F3503226F4503322E86A34228B
:107CC0003F503902F3503226F4503322E86A34220E
:107CD00039AE6FEF3EF03F50335E4050345A40AE05
:107CE000000C3850335E3950345A000C33C03FF02A
:107CF00033503802F4CF32F0F3CF31F03450390240
:107D0000F4CF34F0F3CF33F03802F3503226F4508E
:107D10003322E86A34223F503902F3503226F450BD
:107D20003322E86A3422000C3C6AE7EC3FF03CB6B0
:107D30009EEF3EF03CA20AD03CB403D07F0E346EDE
:107D400019D0800E346E16D0346A14D03CB0FCD7F3
:107D5000870E3560F1D77E0E3564F6D7860E355C1A
:107D600004E0D8903432352AF9D73CA403D0346CDF
:107D700034AEEAD712003C6AE7EC3FF03CB6C5EF00
:107D80003EF03CA20ED03CB405D07F0E346EFF0E08
:107D9000336E1FD0800E346E336A1BD0346A336A60
:107DA00018D03CB0FBD78F0E3560EDD77E0E356412
:107DB000F5D78E0E355C05E0D89034323332352A53
:107DC000F8D73CA406D0336C341EE86A342234AEB3
:107DD000E5D712003C6AE7EC3FF03CB6F4EF3EF02A
:107DE0003CA20FD03CB407D07F0E346EFF0E336E32
:107DF000326E316E25D0800E346E01D0346A000EA2
:107E0000F6D73CB0FBD7316A9F0E3560EBD77E0EBC
:107E10003564F4D79E0E355C07E0D89034323332A7
:107E200032323132352AF6D73CA40AD0316C321EB8
:107E3000331E341EE86A32223322342234AEDED7B7
:107E400012003AEC3FF03CB6000C3CB0010C000CC8
:107E50003AEC3FF03CB6000C3CB0000C3CB4000CDB
:107E6000010C3AEC3FF03CB6000C3CB0000C3CA4DA
:107E7000000C010C3C6AE7EC3FF0FFEC3FF03CB635
:107E800012003CAE08D03CA004D03CA802D03C80FC
:107E900012003C9012003A50355C0BE13950345CD2
:107EA00008E13850335C05E13750325C02E13C8038
:107EB0001200D8A002D03C8E10D035503AC035F018
:107EC0003A6E345039C034F0396E335038C033F024
:107ED000386E325037C032F0376E3A50355C10E0B1
:107EE000FF0F09E03C903CB403D03CAE3C84120050
:107EF0003CAE3C9412003A2AD890393238323732AC
:107F00003750325E3850335A3950345A34BEEAD77B
:107F1000D890323633363436352EF8D7C8D77F0E60
:107F2000356EFF0E346E336E326E12007F0E3CBE25
:107F3000FF0E356E02D07F0E356E800E346E336AC2
:107F4000326AF3D73CAE04D0800E356E346AF7D770
:107F5000356A346AF4D72E502D1040103F10F8E0E7
:107F600030BEF0D72EBE0CD02F503010EBE0D890A2
:107F70003F3640362D362E362F06D8A03006F2D7A3
:107F80003050D4E12F28D2E03FAE11D07F0E3F1405
:107F900002E140A00CD0402AE86A2D222E2207E3FD
:107FA000D8802E322D3240322F2A2F28BFE02F507A
:107FB000C9E040C032F02DC033F02E34346E2F3083
:107FC000356E3432359E3CBE358E95EF3FF03436FB
:107FD000353602E33C843C7E06E13C80356A346AF7
:107FE000336A326A1200352803E0D8803432120036
:107FF000D890343202E13C8212003C8612003936BD
:108000003A3602E33C8C3C7E06E13C883A6A396AA7
:10801000386A376A12003A2803E0D88039321200F1
:10802000D8903932EAE13C8A12000201406B020129
:10803000416B0201426B0201436B0201446B02017E
:108040004E0E3F6F02012D6B1200D9CFE6FFDACF43
:10805000E6FFE1CFD9FFE2CFDAFFE652E652DF6A70
:108060000001FD5130E00001FD6B2CEC1EF0F350DF
:10807000DF6EDF5018E022EC1BF00201446BE66A71
:10808000010EE66EE66AE66A39EC4AF0E552E55220
:10809000E552E5526CC0BDFE6DC0BEFE6EC0BFFEB7
:1080A0006FC0C0FE10D002014451442B03080BE204
:1080B000E66A010EE66EE66AE66AFBEC49F0E55216
:1080C000E552E552E5520E010C5104E10E01010E9C
:1080D000006F05D00E010C5102E00E01006B0E0185
:1080E00018510CE0020EE66EE66AE66AE66AFBEC00
:1080F00049F0E552E552E552E5520ED00E01065127
:108100000BE1020EE66EE66AE66AE66A39EC4AF0D0
:10811000E552E552E552E5520E011E5104E00E0112
:10812000010E026F10D00E0106510DE1040EE66E35
:10813000E66AE66AE66A39EC4AF0E552E552E5524B
:10814000E5520E01026B0E0124510CE0080EE66EA2
:10815000E66AE66AE66AFBEC49F0E552E552E5526A
:10816000E5520ED00E0106510BE1080EE66EE66AEE
:10817000E66AE66A39EC4AF0E552E552E552E55224
:108180000E01125113E00E01065110E00001F451EE
:10819000F5110CE1010EE66EE66AE66AE66AFBECB2
:1081A00049F0E552E552E552E5520ED00E01065176
:1081B0000BE1010EE66EE66AE66AE66A39EC4AF021
:1081C000E552E552E552E5520E012A510CE0100E3F
:1081D000E66EE66AE66AE66AFBEC49F0E552E552CD
:1081E000E552E5520ED00E0106510BE1100EE66E7F
:1081F000E66AE66AE66A39EC4AF0E552E552E5528B
:10820000E5520E01305103E10E01016B09D00E0160
:10821000305106E00E01065103E00E01010E016F20
:10822000376A386A800E396E400E3A6E6CC032F092
:108230006DC033F06EC034F06FC035F031EC3FF0FC
:10824000010A02E0000E01D0010E0E014D6F376AE7
:10825000386AC00E396E400E3A6E6CC032F06DC096
:1082600033F06EC034F06FC035F028EC3FF0010AF7
:1082700002E0000E01D0010E0E01536F376A386A1A
:10828000200E396E420E3A6E6CC032F06DC033F083
:108290006EC034F06FC035F028EC3FF0010A02E008
:1082A000000E01D0010E0E01416F376A386A180EB8
:1082B000396E420E3A6E6CC032F06DC033F06EC053
:1082C00034F06FC035F031EC3FF0010A02E0000EEF
:1082D00001D0010E0E01476F4D0EE66E0E0EE66EDA
:1082E0005EEC33F0E552E552530EE66E0E0EE66E8E
:1082F0005EEC33F0E552E552410EE66E0E0EE66E90
:108300005EEC33F0E552E552470EE66E0E0EE66E79
:108310005EEC33F0E552E5520E014E510BE0400E9B
:10832000E66EE66AE66AE66AFBEC49F0E552E5527B
:10833000E552E5520E0154510EE00E0106510BE1DB
:10834000400EE66EE66AE66AE66A39EC4AF0E55205
:10835000E552E552E5520E0142510BE0800EE66E09
:10836000E66AE66AE66AFBEC49F0E552E552E55258
:10837000E5520E0148510EE00E0106510BE1800E50
:10838000E66EE66AE66AE66A39EC4AF0E552E552DC
:10839000E552E552330EE96E020EEA6EEE5002012E
:1083A00045190CE1EE500201461908E1EE500201B8
:1083B000471904E1EE500201481900E100E033C220
:1083C00045F234C246F235C247F236C248F20E01D7
:1083D00006513DE033C200F034C201F035C202F074
:1083E00036C203F00094010E0116026A036A0050BF
:1083F0000110021003102BE12FC204F030C205F06F
:1084000031C206F032C207F0020E0416056A066A8F
:10841000076A045005100610071019E10E01010E3D
:10842000046FDF5013E0EFEC12F0C1CE32F0C2CE99
:1084300033F0C3CE34F0C4CE35F094EC3EF034507B
:10844000E66EE66A42EC34F0E552E55206D081EC85
:108450000EF032EC34F00E01046B0201492B0201E4
:10846000495164080AE20201496B02014A2B0201E8
:108470004A51020802E202014A6B02014A51020A11
:1084800001E195D0030A4BE0010A01E0EFD0010EB3
:10849000E66E376A386AC80E396E420E3A6EBDCE45
:1084A00032F0BECE33F0BFCE34F0C0CE35F0B6ECF5
:1084B0003DF0BBEC3EF033C000F034C001F000C032
:1084C000E6FF01C0E6FFE66A1DEC46F0E552E55224
:1084D000E552E552010EE66E376A386AC80E396E0B
:1084E000420E3A6EB9CE32F0BACE33F0BBCE34F093
:1084F000BCCE35F0B6EC3DF0BBEC3EF033C000F046
:1085000034C001F000C0E6FF01C0E6FF040EE66ED5
:108510001DEC46F0E552E552E552E552AAD0010EB7
:10852000E66E376A386AC80E396E420E3A6EBDCEB4
:1085300032F0BECE33F0BFCE34F0C0CE35F0B6EC64
:108540003DF0BBEC3EF033C000F034C001F000C0A1
:10855000E6FF01C0E6FFE66A1DEC46F0E552E55293
:10856000E552E552020EE66E376A386A200E396E21
:10857000410E3A6EC1CE32F0C2CE33F0C3CE34F0EB
:10858000C4CE35F0B6EC3DF0BBEC3EF033C000F0AD
:1085900034C001F000C0E6FF01C0E6FF040EE66E45
:1085A0001DEC46F0E552E552E552E55262D030C28C
:1085B00000F0016A00380F0B0F0BEA6A100FE96E2A
:1085C000020EEA22EFCF20F230C200F0016A0F0E55
:1085D0000014EA6A100FE96E020EEA22EFCF21F2D0
:1085E00002012F390F0B0F0BEA6A100FE96E020E12
:1085F000EA22EFCF22F20F0E02012F15EA6A100FC6
:10860000E96E020EEA22EFCF23F234C200F0016AD3
:1086100000380F0B0F0BEA6A100FE96E020EEA2208
:10862000EFCF24F234C200F0016A0F0E0014EA6AA0
:10863000100FE96E020EEA22EFCF25F20201333964
:108640000F0B0F0BEA6A100FE96E020EEA22EFCF52
:1086500026F20F0E02013315EA6A100FE96E020EC0
:10866000EA22EFCF27F20201296B03D048EC47F052
:1086700000D0ACEC45F0DBEC45F089EC34F0E55291
:10868000E552E552E5CFDAFFE7CFD9FF1200D9CFA7
:10869000E6FFDACFE6FFE1CFD9FFE2CFDAFF240E23
:1086A000E12402E3E168E652E16ED950FA0FE96E87
:1086B000FF0EDA20EA6E020EEECFDBFF030EEECFE6
:1086C000DBFF040EEECFDBFF050EEECFDBFFEAD9BA
:1086D000F4D9F8EC4BF0F56E060EE15C02E2E16ACB
:1086E000E552E16EF550E76E0D0EE7CFDBFFDB5094
:1086F000800815E0A2D9376A386A396A3A6A00C038
:1087000032F001C033F002C034F003C035F031EC78
:108710003FF0010A10E1210E0001FE6FFF6B020E17
:10872000DB68030EDB68040EDB687F0EF36E050E5C
:10873000F3CFDBFF66D10D0EDB50050B01E061D1FD
:108740000A0EDBCF00F00B0EDBCF01F0830E00260C
:10875000FF0E012200C0DEFF01C0DDFFD950060F71
:1087600067D978D9DF50010B0FE0DF06010E01E277
:10877000DB06D950180F5CD9D890EF36010EEB36D6
:10878000020EEB36030EEB36D9CFE9FFDACFEAFF64
:10879000020E386E396AEECF33F0EDCF34F023ECB1
:1087A0003EF033C0EEFF34C0EDFF140EDB6A150E51
:1087B000DB6A160EDB6A170EDB6A1C0EDB6A1D0E07
:1087C000DB6A1E0EDB6A010EF36E1F0EF3CFDBFFBA
:1087D000010EF36E0E0EF3CFDBFF0F0EDB6A0E0EF3
:1087E000DBCF00F00F0EDBCF01F0D890015004E694
:1087F0001A0E005C000E015801E398D0180EDBCF72
:1088000000F0190EDBCF01F01A0EDBCF02F01B0EC9
:10881000DBCF03F0010E1F0B07E0D89000360136C6
:1088200002360336E806F9E1180E00C0DBFF190E28
:1088300001C0DBFF1A0E02C0DBFF1B0E03C0DBFF13
:10884000140EDBCF08F0150EDBCF09F0160EDBCFD0
:108850000AF0170EDBCF0BF0010E1F0B07E0D890CC
:10886000083609360A360B36E806F9E1D9501C0FEE
:10887000DFD80850EE24046E0950EE20056E0A5031
:10888000EE20066E0B50EE20076ED950180FD0D890
:108890000450EE5C006E0550EE58016E0650EE5826
:1088A000026E0750EE58036E200E00C0DBFF210E53
:1088B00001C0DBFF220E02C0DBFF230E03C0DBFF83
:1088C000200EDBCF32F0210EDBCF33F0220EDBCFD8
:1088D00034F0230EDBCF35F03534000E351809E6C1
:1088E000D880000E3254000E3354000E3454000E63
:1088F000355411E2D950200F9BD8ACD8DAD81C0ED1
:10890000DB50EE121D0EDB50EE121E0EDB50EE128F
:108910001F0EDB50EE12D9501C0F8AD8B1D80E0EA4
:10892000DB2A0F0E01E25BD7DB2A59D7CBD8100E1A
:1089300000C0DBFF110E01C0DBFF180EDBCF33F0F0
:10894000190EDBCF34F0120E33C0DBFF130E34C030
:10895000DBFFAFD895D8D950100F6AD8EE50ED1084
:1089600012E0D950120F64D8EE50ED1006E1AAD8EB
:10897000005001100210031006E09BD8EE2A000EF2
:10898000EE22EE22EE220C0EDB6A93D8060EEECF1C
:10899000DBFF070EEECFDBFF080EEECFDBFF090E8D
:1089A000EECFDBFF7E0EF36E0A0EF3CFDBFF0B0E76
:1089B000DB6AD950020FE66E000EDA20E66E72D83E
:1089C00086EC4CF0E552E552E552E552DECFE6FF8B
:1089D000DDCFE6FF72D85AEC4BF0F56E060EE15C87
:1089E00002E2E16AE552E16EF550020E31C0DBFFB2
:1089F000030E32C0DBFF040E33C0DBFF050E34C0B4
:108A0000DBFF1BD800C031F001C032F002C033F0F0
:108A100003C034F0F56E240EE15C02E2E16AE55237
:108A2000E16EF550E552E5CFDAFFE7CFD9FF12004E
:108A3000E96E000EDA20EA6E1200020EDBCF00F0C3
:108A4000030EDBCF01F0040EDBCF02F0050EDBCF0F
:108A500003F01200180EEECFDBFF190EEECFDBFF96
:108A60001A0EEECFDBFF1B0EEECFDBFF1200EECFB8
:108A7000E6FFEECFE6FFEECFE6FFEFCFE6FF120018
:108A8000D890030EEB32020EEB32010EEB32EF32D6
:108A90001200EE500016EE500116EE500216EE5087
:108AA00003161200D950060FE66E000EDA20E66EAD
:108AB0001200D950140F18EF45F0D950020FB8DF4B
:108AC00037EF45F0010E006E016A026A036AF1DFBA
:108AD00049EF45F0D9CFE6FFDACFE6FFE1CFD9FF86
:108AE000E2CFDAFFE65202012D0500E00201296B18
:108AF0000201040E2A6F0201070E2B6F0201010E04
:108B00002C6F0201010E2D6FDF6ADFCF00F0080E1F
:108B1000E76E0018E8AE02D0E73402D0E750005C00
:108B20000CE2DFCFE9FFEA6AE9BEEA68200EE92637
:108B3000020EEA22EF6ADF2AE8D70201286B3BD84F
:108B40000BD8010EF36EF46A00D0E552E552E5CF82
:108B5000DAFFE7CFD9FF1200D9CFE6FFDACFE6FF81
:108B6000E1CFD9FFE2CFDAFFE652DF6ADFCF00F0D4
:108B7000080EE76E0018E8AE02D0E73402D0E750E6
:108B8000005C12E2DFCFE9FFEA6AE9BEEA68200E84
:108B9000E926020EEA22EF50E66EDF28E66E2FD8B5
:108BA000E552E552DF2AE2D7E552E552E5CFDAFF9A
:108BB000E7CFD9FF120029C2E6FF090EE66E1FD8E3
:108BC000E552E5522AC2E6FF0A0EE66E18D8E552D3
:108BD000E5522BC2E6FF0B0EE66E11D8E552E552C8
:108BE0002CC2E6FF0C0EE66E0AD8E552E5522DC205
:108BF000E6FF0F0EE66E03D8E552E5521200D9CF1C
:108C0000E6FFDACFE6FFE1CFD9FFE2CFDAFFE652A7
:108C10008598FD0EDBCFE6FF45EC51F0E552FC0EEA
:108C2000DBCFE6FF45EC51F0E5528588E552E55291
:108C3000E5CFDAFFE7CFD9FF1200D9CFE6FFDACFD1
:108C4000E6FFE1CFD9FFE2CFDAFFE652FB0EDBCF42
:108C500000F0FC0EDBCF01F00001800E011442E1B8
:108C6000FB0EDBCF00F0FC0EDBCF01F0013404E2A1
:108C700000500F08270E01540AE20F0EF36EFB0E90
:108C8000F3CFDBFF270EF36EFC0EF3CFDBFFFB0E03
:108C9000DBCF00F0FC0EDBCF01F0E80E386E030EE8
:108CA000396E00C033F001C034F023EC3EF033C025
:108CB00000F034C001F00A0E386E396A00C033F09B
:108CC00001C034F023EC3EF02FC000F030C001F0C2
:108CD000FD0EDB50EA6A200FE96E020EEA2200C0A8
:108CE000EFFF21D0FB0EDBCF00F0FC0EDBCF01F05D
:108CF000D880015004E7190E005CFC0E01580AE20E
:108D0000190EF36EFB0EF3CFDBFFFC0EF36EFC0EC1
:108D1000F3CFDBFFFD0EDB50EA6A200FE96E020E97
:108D2000EA22010EEF6EFB0EDBCF00F0FC0EDBCF74
:108D300001F0640E386E396A00C033F001C034F0BF
:108D400023EC3EF033C000F034C001F00A0E386E60
:108D5000396A00C033F001C034F023EC3EF02FC07C
:108D600000F030C001F0FD0EDB28EA6A200FE96E4A
:108D7000020EEA2200C0EFFFFB0EDBCF00F0FC0E7C
:108D8000DBCF01F00A0E386E396A00C033F001C043
:108D900034F023EC3EF033C000F034C001F00A0E92
:108DA000386E396A00C033F001C034F023EC3EF075
:108DB0002FC000F030C001F0FD0EDB50020FEA6A58
:108DC000200FE96E020EEA2200C0EFFFFB0EDBCFA0
:108DD00000F0FC0EDBCF01F00A0E386E396A00C0DD
:108DE00033F001C034F023EC3EF02FC000F030C06F
:108DF00001F0FD0EDB50030FEA6A200FE96E020E50
:108E0000EA2200C0EFFFDF6AFA0EDB50DF5C18E2F7
:108E1000FD0EDB50DF24EA6A200FE96E020EEA2223
:108E2000EF500BE1FD0EDB50DF24EA6A200FE96E04
:108E3000020EEA220F0EEF6E01D002D0DF2AE4D735
:108E4000FA0EDBCF00F0040EE76E0018E8AE02D099
:108E5000E73402D0E750005C0DE2FA0EDBCFE6FF0C
:108E6000FD0EDB50E552E724EA6A200FE96E020EA0
:108E7000EA22EF8E02012969E552E552E5CFDAFFD9
:108E8000E7CFD9FF120002012D6B02012969120000
:108E9000D9CFE6FFDACFE6FFE1CFD9FFE2CFDAFFA5
:108EA000E65202012D6BDF6A080EDF5C09E2DF503B
:108EB000EA6A200FE96E020EEA22EF6ADF2AF4D78F
:108EC0000201296BE552E552E5CFDAFFE7CFD9FF82
:108ED00012003DD8F3CF00F0F4CF01F000500110A4
:108EE00012E1010EE66EE66AE66AE66A73EC49F0A4
:108EF000E552E552E552E5520201376B386BC80E78
:108F0000396F420E3A6F1F0E006E580E016E026AE4
:108F100000C0E6FF01C0E6FF7AEC04F0E552E5523E
:108F200037C2E6FF38C2E6FF39C2E6FF3AC2E6FFC3
:108F3000740EE66E000EE66E74EC3BF0F56E060EF7
:108F4000E15C02E2E16AE552E16EF5501200D9CF30
:108F5000E6FFDACFE6FFE1CFD9FFE2CFDAFFE65254
:108F6000E652E652E652010E006E580E016E026A9B
:108F700000C0E6FF01C0E6FF7AEC04F0E552E552DE
:108F8000060EE66EE66A370EE66E020EE66E000E1E
:108F9000E66EE66A9FEC4AF0F56E060EE15C02E2D0
:108FA000E16AE552E16EF550000EE66EE66A040EE7
:108FB000E66EE66A370EE66E020EE66E13EC4DF0D4
:108FC000F56E060EE15C02E2E16AE552E16EF550F3
:108FD000F3CF3DF2F4CF3EF2020EDB6A030EDB6A02
:108FE000020EDBCF00F0030EDBCF01F0060E005CBB
:108FF000000E01583AE2020EDBCFE9FF030EDBCF91
:10900000EAFF370EE926020EEA22EF50E66EE66A24
:10901000020EDBCFE6FF030EDBCFE6FFE80E006EAD
:10902000570E016E026A00C0E6FF01C0E6FF02C0F3
:10903000E6FF740EE66E000EE66E0FEC4EF0F56E77
:10904000090EE15C02E2E16AE552E16EF550740E50
:10905000E66E000EE66E53EC04F0E552E552020EA9
:10906000DB2A030E01E3DB2ABBD73DC2E6FF3EC28B
:10907000E6FFDA0E006E570E016E026A00C0E6FFD0
:1090800001C0E6FF02C0E6FF740EE66E000EE66E5B
:109090000FEC4EF0F56E070EE15C02E2E16AE5527C
:1090A000E16EF550740EE66E000EE66E53EC04F0C1
:1090B000E552E55202013B5102013D1904E1020172
:1090C0003C5102013E1911E0BE0E006E570E016EBA
:1090D000026A00C0E6FF01C0E6FF7AEC04F0E55248
:1090E000E552F36AF46A12D011D0A20E006E570E48
:1090F000016E026A00C0E6FF01C0E6FF7AEC04F0F0
:10910000E552E552010EF36EF46A00D0F56E040EDE
:10911000E15C02E2E16AE552E16EF550E552E5CF2D
:10912000DAFFE7CFD9FF1200D9CFE6FFDACFE6FFAB
:10913000E1CFD9FFE2CFDAFFE652E652850E006EAC
:10914000570E016E026A00C0E6FF01C0E6FF7AEC2E
:1091500004F0E552E552000EE66EE66A040EE66E95
:10916000E66A370EE66E020EE66E13EC4DF0F56E13
:10917000060EE15C02E2E16AE552E16EF550F3CFE2
:109180003BF2F4CF3CF23BC2E6FF3CC2E6FF040EEA
:10919000E66EE66A060EE66EE66A560E006E570E3C
:1091A000016E026A00C0E6FF01C0E6FF02C0E6FFF2
:1091B000740EE66E000EE66E0FEC4EF0F56E0B0EC2
:1091C000E15C02E2E16AE552E16EF550740EE66E92
:1091D000000EE66E53EC04F0E552E552DE6ADD6AFD
:1091E000DECF00F0DDCF01F0060E005C000E01586E
:1091F00035E2DECFE9FFDDCFEAFF370EE926020ECA
:10920000EA22EF50E66EE66ADECFE6FFDDCFE6FF4C
:10921000E80E006E570E016E026A00C0E6FF01C044
:10922000E6FF02C0E6FF740EE66E000EE66E0FEC7F
:109230004EF0F56E090EE15C02E2E16AE552E16E84
:10924000F550740EE66E000EE66E53EC04F0E55237
:10925000E552DF2A010E01E3DB2AC2D7060EE66ED5
:10926000E66A370EE66E020EE66E000EE66EE66AFF
:1092700017EC4BF0F56E060EE15C02E2E16AE55296
:10928000E16EF550010EF36EF46A00D0E552E5523E
:10929000E552E5CFDAFFE7CFD9FF1200D9CFE6FFDD
:1092A000DACFE6FFE1CFD9FFE2CFDAFFE652E652AE
:1092B000E652E652E65202012F6B306B316B326B95
:1092C0000201336B346B356B366BF56E050EE15C6A
:1092D00002E2E16AE552E16EF550E552E5CFDAFFD0
:1092E000E7CFD9FF1200D9CFE6FFDACFE6FFE1CF13
:1092F000D9FFE2CFDAFFD950FA0FE96EFF0EDA207C
:10930000EA6E02012F51EE14006E02013051EE148C
:10931000016E02013151EE14026E02013251EE145F
:10932000036E005001100210031013E1FA0EDB501F
:1093300002012F13FB0EDB5002013013FC0EDB5039
:1093400002013113FD0EDB5002013213010E03D076
:1093500002D0000E00D0E552E5CFDAFFE7CFD9FF0B
:109360001200D9CFE6FFDACFE6FFE1CFD9FFE2CF97
:10937000DAFFD950FA0FE96EFF0EDA20EA6E020129
:109380002F51EE14006E02013051EE14016E0201F5
:109390003151EE14026E02013251EE14036E005090
:1093A0000110021003101FE0FA0EDBCF00F0FB0EDD
:1093B000DBCF01F0FC0EDBCF02F0FD0EDBCF03F0C4
:1093C000001E011E021E031E005002012F17015035
:1093D0000201301702500201311703500201321707
:1093E000010E03D002D0000E00D0E552E5CFDAFF27
:1093F000E7CFD9FF1200D9CFE6FFDACFE6FFE1CF02
:10940000D9FFE2CFDAFFD950FA0FE96EFF0EDA206A
:10941000EA6E02013351EE14006E02013451EE1473
:10942000016E02013551EE14026E02013651EE1446
:10943000036E005001100210031013E1FA0EDB500E
:1094400002013313FB0EDB5002013413FC0EDB5020
:1094500002013513FD0EDB5002013613010E03D05D
:1094600002D0000E00D0E552E5CFDAFFE7CFD9FFFA
:109470001200D9CFE6FFDACFE6FFE1CFD9FFE2CF86
:10948000DAFFD950FA0FE96EFF0EDA20EA6E020118
:109490003351EE14006E02013451EE14016E0201DC
:1094A0003551EE14026E02013651EE14036E005077
:1094B0000110021003101FE0FA0EDBCF00F0FB0ECC
:1094C000DBCF01F0FC0EDBCF02F0FD0EDBCF03F0B3
:1094D000001E011E021E031E005002013317015020
:1094E00002013417025002013517035002013617EA
:1094F000010E03D002D0000E00D0E552E5CFDAFF16
:10950000E7CFD9FF1200D9CFE6FFDACFE6FFE1CFF0
:10951000D9FFE2CFDAFFE652DF6AAA6AFD0EDB501E
:10952000A96EA69EA69CA680A850DF6EDF5000D034
:10953000E552E552E5CFDAFFE7CFD9FF1200D9CFE8
:10954000E6FFDACFE6FFE1CFD9FFE2CFDAFFE6525E
:10955000E652DE6ADD6AF80EDBCF00F0DB06F90EBC
:10956000DBCF01F001E2DB06005001101FE0FC0E32
:10957000DBCF00F0DB2AFD0EDBCF01F001E3DB2ABD
:109580000050E66EC0DFE552E66EFA0EDBCFE9FF73
:10959000DB2AFB0EDBCFEAFF01E3DB2AE552E750D3
:1095A000EF6EDF2A010E01E3DB2AD5D7DF5000D0B2
:1095B000E552E552E552E5CFDAFFE7CFD9FF1200D9
:1095C000D9CFE6FFDACFE6FFE1CFD9FFE2CFDAFF6E
:1095D000E652F250800B01E0010EDF6EAA6AFC0E2B
:1095E000DB50A96EFB0EDB50A86EA69EA69CA6843F
:1095F000A198F29E550EA76EAA0EA76EA682DF5006
:10960000E8B0F28EE8A0F29EDF68A1A806D0DF5095
:10961000DF06000901E101D0F8D7A694A6B2FED773
:10962000E552E552E5CFDAFFE7CFD9FF1200D9CFF7
:10963000E6FFDACFE6FFE1CFD9FFE2CFDAFFE6526D
:10964000E652DE6ADD6AF80EDBCF00F0DB06F90ECB
:10965000DBCF01F001E2DB060050011021E0FA0E41
:10966000DBCFE9FFDB2AFB0EDBCFEAFF01E3DB2ADE
:10967000EF50E66EFC0EDBCF00F0DB2AFD0EDBCFF9
:1096800001F001E3DB2A00C0E6FF01C0E6FF98DF3E
:10969000E552E552E552DF2A010E01E3DB2AD3D77A
:1096A000DF5000D0E552E552E552E5CFDAFFE7CFD3
:1096B000D9FF120098D8E1CFD9FFE2CFDAFF0C0E24
:1096C000E12402E3E168E652E16ED950FA0FE96E57
:1096D000FF0EDA20EA6E080EEECFDBFF090EEECFAA
:1096E000DBFF0A0EEECFDBFF0B0EEECFDBFF7BD8EE
:1096F000D950080FE96E000EDA20EA6EEECFE6FFD1
:10970000EECFE6FFEECFE6FFEFCFE6FFF8EC4BF053
:10971000F56E060EE15C02E2E16AE552E16EF5509B
:10972000E76E070EE7CFDBFFDB50840B3AE1070E55
:10973000DB041AE1060EDB5006E0006A016A026AE9
:10974000800E036E04D0006A016A026A036A080E82
:1097500000C0DBFF090E01C0DBFF0A0E02C0DBFF09
:109760000B0E03C0DBFF1DD0F80EDBCF00F0F90EAF
:10977000DBCF01F0D950040FE96E000EDA20EA6E5B
:109780000050EE260150ED22D950080FE66E000E73
:10979000DA20E66E28D886EC4CF0E552E552E55228
:1097A000E552080EDBCF00F0090EDBCF01F00A0E08
:1097B000DBCF02F00B0EDBCF03F000C031F001C0B5
:1097C00032F002C033F003C034F0F56E0C0EE15CF1
:1097D00002E2E16AE552E16EF550E552E5CFDAFFCB
:1097E000E7CFD9FF1200D9CFE6FFDACFE6FF1200AC
:1097F000D9CFE6FFDACFE6FFE1CFD9FFE2CFDAFF3C
:10980000E652006801687F0E026E036AD950FA0FB3
:10981000E96EFF0EDA20EA6EEE500016EE500116E9
:10982000EE500216EE5003166AD800C0EEFF01C0DB
:10983000EEFF02C0EEFF03C0EEFFFD0EDB50800B1B
:1098400002E0010E01D0000EE66E59D8060EE926A0
:10985000000EEA22E552E750EF6EFC0EDBCF00F07F
:10986000FD0EDBCF01F0D89000360136FC0E00C0B3
:10987000DBFFFD0E01C0DBFFDB50E66E40D8040EBF
:10988000E926000EEA22E552E750EE6EED6AFD0E83
:10989000DB50006E016AFF0E001818E1015016E15E
:1098A0002ED8EECF00F0EECF01F0EECF02F0EFCFEA
:1098B00003F0005001100210031006E0210E000119
:1098C000FE6FFF6B800E0BD0040E09D0FD0EDB5037
:1098D00008E115D8EE6AEE6AEE6AEE6A010EDF6EF6
:1098E00006D0020EDF6E0BD8EE52EE52EE8EDF5037
:1098F000E552E552E5CFDAFFE7CFD9FF1200F80EC7
:10990000DBCFE9FFF90EDBCFEAFF1200D9CFE6FF8C
:10991000DACFE6FFE1CFD9FFE2CFDAFF5BD801343F
:1099200011E20050FE08000E01540CE276D805E06A
:109930006CD8800EEE6EEE6847D067D8800EEE6E63
:109940007F0E0ED047D8D890015004E6010E005C7F
:10995000000E01580BE261D805E057D8EE6A800E80
:10996000EE6E32D052D8EE6AEE6A2ED047D8EECFE5
:1099700000F0EECF01F0EECF02F0EFCF03F032D8DF
:1099800000C0EEFF01C0EEFF02C0EEFF03C0EEFF1D
:1099900021D80050010B05E025D8020E3AD8EF8EF1
:1099A00004D020D8020E35D8EF9E14D8D8900132BA
:1099B000003218D8030E2DD800C0EFFF1AD804E0EB
:1099C00011D8030E26D8EF8EE552E5CFDAFFE7CFA8
:1099D000D9FF120013D8040E1CD8EECF00F0EFCF41
:1099E00001F01200FA0EDBCFE9FFFB0EDBCFEAFF3E
:1099F000120004D8060E0DD8EF501200FC0EDBCF7B
:109A0000E9FFFD0EDBCFEAFF1200ECDFEE6AEE6A43
:109A10001200E926000EEA221200220E0001FE6F5B
:109A2000FF6BF9EF4CF0D9CFE6FFDACFE6FFE1CFDD
:109A3000D9FFE2CFDAFFE652E652E652E652E652AC
:109A4000F80EDBCFDEFFDBCFDDFFFA0EDBCF00F061
:109A5000DB06FB0EDBCF01F001E2DB06005001105C
:109A600052E0DECF00F0DDCF01F001C000F0016A6E
:109A7000FC0EDBCFE9FFFD0EDBCFEAFFEF50001855
:109A8000E76E020EE7CFDBFF020EE66EE66A020E1D
:109A9000016ADB34FE0B0136006EF00E0026050E67
:109AA0000122026A00C0E6FF01C0E6FF02C0E6FF35
:109AB000D950030FE66E000EDA20E66E63EC01F07B
:109AC000F56E070EE15C02E2E16AE552E16EF550E7
:109AD000DFCF02F002C003F0026A000E0216FF0E92
:109AE0000316030EDB500218006E040EDB50031841
:109AF000016E00C0DEFF01C0DDFFFC0EDB2AFD0EA3
:109B000001E3DB2AA2D7DECF00F0DDCF01F000C0F9
:109B1000F3FF01C0F4FF00D0F56E050EE15C02E238
:109B2000E16AE552E16EF550E552E5CFDAFFE7CFA5
:109B3000D9FF1200FF0EE3CFEAFFE552FF0EE3CF9D
:109B4000E9FFE552E66AE66AD9CFE6FFDACFE6FF3B
:109B5000FC0EE124D96EFF0EE220DA6EE66AE66AB8
:109B6000E66A200EEF5C06E0090EEF5C03E0EF66AC
:109B700003D03FD0EE50F5D72D0EEF5C03E1FF0E82
:109B8000E32A03D02B0EEF5C01E1EE502F0EEF64C1
:109B900024D03A0EEF6021D0D890F90EE336FA0EB9
:109BA000E336FD0EDECFE3FFFE0EDDCFE3FFD89000
:109BB000F90EE336FA0EE336D890F90EE336FA0ED4
:109BC000E336FD0EE350DE26FE0EE350DD22300EBE
:109BD000EE5CDE26000EDD22D9D7FF0EE3CFE8FFD4
:109BE000E85207E0F90EE31EE32AFA0ED8B4E306C2
:109BF000E31EE552E552E552FF0EE3CFDAFFE552F0
:109C0000FF0EE3CFD9FFE552E1CFE9FFE2CFEAFF54
:109C1000ED52ED52EECFF3FFEFCFF4FF1200D9CFAC
:109C2000E6FFDACFE6FFE1CFD9FFE2CFDAFFE65277
:109C3000E652E652E652D950F90F006EFF0EDA20D6
:109C4000016E020E00C0DBFF030E01C0DBFF020E3F
:109C5000DBCFE6FF030EDBCFE6FFF90EDBCFE6FF3F
:109C6000FA0EDBCFE6FFFB0EDBCFE6FFD950FC0F91
:109C7000E66EFF0EDA20E66EECEC14F0F56E070EE1
:109C8000E15C02E2E16AE552E16EF550F3CFDEFFFE
:109C9000F4CFDDFFFC0EDBCFE9FFFD0EDBCFEAFFEB
:109CA000EF6ADECF00F0DDCF01F000C0F3FF01C0AE
:109CB000F4FFF56E040EE15C02E2E16AE552E16E4A
:109CC000F550E552E5CFDAFFE7CFD9FF1200300EAD
:109CD000F66E080EF76E000EF86E01010900F550E1
:109CE000F86F0900F550F96F03E1F86701D03DD036
:109CF0000900F550F36F0900F550F46F0900F550B5
:109D0000F56F09000900F550E96E0900F550EA6E9B
:109D1000090009000900F550F66F0900F550F76FCA
:109D200009000900F6CFFAF1F7CFFBF1F8CFFCF10B
:109D3000F3C1F6FFF4C1F7FFF5C1F8FF0101F653D7
:109D400002E1F75307E00900F550EE6EF607F8E27E
:109D5000F707F9D7FAC1F6FFFBC1F7FFFCC1F8FF1F
:109D60000101F807000EF95BBFD71200D9CFE6FF5B
:109D7000DACFE6FFE1CFD9FFE2CFDAFFFB0EDBCF90
:109D800000F0FC0EDBCF01F00001800E01141AE19F
:109D9000FB0EDBCFE9FFFC0EDBCFEAFFEECFF3FFDC
:109DA000EDCFF4FFEE2A000EEF22F3CFE9FFF4CF60
:109DB000EAFFFD0EDBCFEFFFEF50016AF36E01C04B
:109DC000F4FF10D0FB0EDB50FE0806E1FD0EDBCFEA
:109DD000E6FFEDEC51F005D0FD0EDBCFE6FF15EC14
:109DE00052F0E552E552E5CFDAFFE7CFD9FF120096
:109DF00031503602F3CF2DF0F4CF2EF03702F3506E
:109E00002E26000EF4202F6E31503802F3502F26EC
:109E1000000EF420306E31503902F35030263250AB
:109E20003602F3502E26F4502F22000E30223250EC
:109E30003702F3502F26F450302232503802F350BC
:109E4000302633503602F3502F26F4503022335050
:109E50003702F350302634503602F35030261200C9
:109E6000FE0EE3CFE9FFFF0EE3CFEAFFF36AF46AE9
:109E7000EE5203E0F34AF42AFBD71200FF0EE3CFC1
:109E8000F8FFE552FF0EE3CFF7FFE552FF0EE3CFF9
:109E9000F6FFE552E66AE66AE66A0900F55209E06D
:109EA000FD0EE32A05E1FE0EE32A02E1FF0EE32A9E
:109EB000F4D7FD0EE3CF32F0FE0EE3CF33F0FF0E0A
:109EC000E3CF34F01200D9CFE6FFDACFE6FFE1CFDF
:109ED000D9FFE2CFDAFF3F0EC716C66AFD0EDB5090
:109EE000C612FB0EDB50C712FC0EDB50030A09E062
:109EF000010A04E0020A06E1C78C04D0C78CC688B8
:109F000001D0C688FD0EDB50050A03E0010A04E11A
:109F1000928A9486C79E01D09496949A9488C68A11
:109F2000E552E5CFDAFFE7CFD9FF1200D9CFE6FF40
:109F3000DACFE6FFE1CFD9FFE2CFDAFFE652E65211
:109F4000D950FD0F006EFF0EDA2000C0DEFFDD6E7F
:109F5000DECFE9FFDDCFEAFFEF9EFA0EDBCF00F0A8
:109F6000FB0EDBCF01F0FC0EDBCF02F0FD0EDBCFF2
:109F700003F000C031F001C032F002C033F003C082
:109F800034F0E552E552E552E5CFDAFFE7CFD9FFED
:109F90001200D9CFE6FFDACFE6FFE1CFD9FFE2CF5B
:109FA000DAFF6C6A6B6AFD0EDBB06C88DBA202D054
:109FB0006C8C6B8CDBB46C8EDBA602D06B8801D012
:109FC0006B8ADBA802D06C8401D06C94DBAC02D02D
:109FD000A38A01D0A39ADBAE02D0A38801D0A398B4
:109FE000FC0EDB506F6E6C8A6B8EE552E5CFDAFFAC
:109FF000E7CFD9FF1200D9CFE6FFDACFE6FFE1CFF6
:10A00000D9FFE2CFDAFFAC6AAB6AFD0EDBB0AC88F9
:10A01000DBA202D0AC8CAB8CDBB4AC8EDBA602D066
:10A02000AB8801D0AB8ADBA802D0AC8401D0AC9461
:10A03000DBAC02D09D8A01D09D9ADBAE02D09D8818
:10A0400001D09D98FC0EDB50AF6EAC8AAB8EE55212
:10A05000E5CFDAFFE7CFD9FF1200D9CFE6FFDACF9D
:10A06000E6FFE1CFD9FFE2CFDAFFE652E652DF6A40
:10A07000FB0EDB50DF5C18E2A4AAFED7D0EC50F058
:10A08000E76E010EE7CFDBFFFC0EDBCFE9FFFD0E35
:10A09000DBCFEAFF010EDBCFEFFFFC0EDB2AFD0E6C
:10A0A00001E3DB2ADF2AE4D7E552E552E552E5CFAA
:10A0B000DAFFE7CFD9FF1200D9CFE6FFDACFE6FF0C
:10A0C000E1CFD9FFE2CFDAFFE652E652FC0EDBCF5A
:10A0D00000F0FD0EDBCF01F0060ED8900036013601
:10A0E000E804FBE100C0DEFF01C0DDFF010EDB5034
:10A0F000BB6EDF50E840E8403F0B300B006ECF0EE8
:10A10000BA140010BA6EE552E552E552E5CFDAFF17
:10A11000E7CFD9FF1200306A2F6A2E6A2D6A200E0F
:10A12000E76ED89031363236333634362D362E3609
:10A130002F36303636502D5C37502E5838502F5829
:10A140003950305809E336502D5E37502E5A38506A
:10A150002F5A3950305A312AE72EE4D71200D9CF7E
:10A16000E6FFDACFE6FFE1CFD9FFE2CFDAFFFD0E5F
:10A17000DB507E0BCD6EFD0EDBAC02D0CD8E01D060
:10A18000CD9ECF6ACE6A9E90DBAE02D09D8001D07C
:10A190009D90CD80E552E5CFDAFFE7CFD9FF1200E1
:10A1A000D9CFE6FFDACFE6FFE1CFD9FFE2CFDAFF82
:10A1B000E652F20E0E01F3176BAC03D0F3916BB0C5
:10A1C000F3816BB4F3856BB2F3876E50DF6EDF50B3
:10A1D000E552E552E5CFDAFFE7CFD9FF1200D9CF3C
:10A1E000E6FFDACFE6FFE1CFD9FFE2CFDAFF0C0ED0
:10A1F000BA6EB1B607D0CA94FD0EDB50CB6E949206
:10A20000CA8406D07694FD0EDB50776E94927684E5
:10A21000E552E5CFDAFFE7CFD9FF1200D9CFE6FF4D
:10A22000DACFE6FFE1CFD9FFE2CFDAFFE652E6521E
:10A23000FC0EDBCFDEFFDBCFDDFF010EDB50CF6E90
:10A24000DF50CE6EE552E552E552E5CFDAFFE7CFBB
:10A25000D9FF1200D9CFE6FFDACFE6FFE1CFD9FF71
:10A26000E2CFDAFFFD0EDB50FB0BCA6ECC6A9E928A
:10A27000FD0EDBAE02D09D8201D09D92CA84E552D4
:10A28000E5CFDAFFE7CFD9FF1200D9CFE6FFDACF6B
:10A29000E6FFE1CFD9FFE2CFDAFFFD0EDB50C96E5A
:10A2A000C6AE02D0FF0E03D0C7A0FED7000EE55207
:10A2B000E5CFDAFFE7CFD9FF1200FF0EE350436E80
:10A2C000EF0E01D0F30EE76EE72E64EF51F00C0EA7
:10A2D000426EE76AE72E6AEF51F0422E69EF51F0C5
:10A2E000432E62EF51F01200D9CFE6FFDACFE6FF3E
:10A2F000E1CFD9FFE2CFDAFF6CAC04D06C900E0155
:10A30000F3B36C80FD0EDB506D6EE552E5CFDAFFE6
:10A31000E7CFD9FF1200D9CFE6FFDACFE6FFE1CFD2
:10A32000D9FFE2CFDAFFACAC04D0AC900101FDB3B1
:10A33000AC80FD0EDB50AD6EE552E5CFDAFFE7CF26
:10A34000D9FF1200306A2F6A100EE76ED8903336AC
:10A3500034362F36303638502F5C3950305805E3BC
:10A3600038502F5E3950305A332AE72EF0D712007A
:10A370003E0EE66E2AEC51F0E5525F0EE66EEFEC13
:10A3800050F0E552C00EE66EE66A5CEC50F0E55225
:10A39000E55294821200F36AF46AFF0EE124E96E3A
:10A3A000FF0EE220EA6EED6607D02F0EEF6404D0B8
:10A3B0003A0EEF6001D0F32A1200FF0EE350436E15
:10A3C000480E01D04C0EE76EE72EFED7E76AE72E67
:10A3D000FED7432EF7D700001200FF0EE350ACBAB1
:10A3E00004D0AF6AAB8EAC8A949CACA2FED7AD6EA3
:10A3F000F36EF46A12001DEE00F02DEE00F0F86A24
:10A400003C9C67EC4EF018EC39F0FDD7120030316F
:10A41000323334353637383961626364656600FF3C
:10A42000C96AC7A0FED7C950120012000000000080
:10A430000000F016C83E9638F2B8963872B9D86364
:10A440001C3E0000003F50000400020064000000B9
:10A450000000FFFFFA0000000000000000007E3056
:10A460006D79335B5F707F7B771F4E3D4F47FF00F9
:10A47000FF00FF00FF00FF00FF00FF00FF00FF00E4
:10A48000FF00FF00FF00FF00FF00FF00FF00FF00D4
:10A49000FF00FF00FF00FF00FF00FF00FF00FF00C4
:10A4A000FF00FF00FF00FF00FF00FF00FF00FF00B4
:020000040001F9
:10FFF000000058013005062024005301FF00421A7A
:020000040030CA
:0E0000000022020E83018100FF80FFA0FF405E
:020000040020DA
:08000000FFFFFFFFFFFFFFFF00
:0200000400F00A
:10000000CEFFC742D839FFFFFFFFFFFFFFFFFFFF13
:10001000FFFFFFFFFFFFFFFFFFFFFFFFFFFFFFFFF0
:10002000FFFFFFFFFFFFFFFFFFFFFFFFFFFFFFFFE0
:10003000FFFFFFFFFFFFFFFFFFFFFFFFFFFFFFFFD0
:10004000500004000200000000000000FCFF050159
:10005000A5A4FFFFFFFFFFFFFFFFFFFFFFFFFFFF65
:10006000500004000200000000000000FCFF050139
:10007000A5A4FFFFFFFFFFFFFFFFFFFFFFFFFFFF45
:10008000FFFFFFFFFFFFFFFFFFFFFFFFFFFFFFFF80
:10009000FFFFFFFFFFFFFFFFFFFFFFFFFFFFFFFF70
:1000A000FFFFFFFFFFFFFFFFFFFFFFFFFFFFFFFF60
:1000B000FFFFFFFFFFFFFFFFFFFFFFFFFFFFFFFF50
:00000001FF
